:020000022000DC
:1070000000000420B5720200DD720200DF7202008F
:10701000E1720200E3720200E5720200000000006B
:10702000000000000000000000000000E772020005
:10703000E972020000000000EB720200ED72020033
:1070400091B40200EF720200FDBD0200EF72020077
:10705000EF720200EF72020095B80200EF720200B8
:10706000EF720200EF720200EF720200EF72020094
:10707000EF720200EF720200EF720200EF72020084
:10708000EF7202007D910200EF720200EF720200C7
:10709000EF720200EF72020079CB0200EF72020081
:1070A000EF720200EF720200EF720200EF72020054
:1070B000EF720200EF72020000000000000000000A
:1070C000EF720200EF720200EF720200EF72020034
:1070D000EF720200EF720200EF720200EF72020024
:1070E000EF720200EF720200EF7202000000000077
:1070F00000000000EF72020000000000EF720200CA
:10710000000000000000000000000000000000007F
:10711000000000000000000000000000000000006F
:10712000000000000000000000000000000000005F
:10713000000000000000000000000000000000004F
:10714000000000000000000000000000000000003F
:10715000000000000000000000000000000000002F
:10716000000000000000000000000000000000001F
:10717000000000000000000000000000000000000F
:1071800000000000000000000000000000000000FF
:1071900000000000000000000000000000000000EF
:1071A00000000000000000000000000000000000DF
:1071B00000000000000000000000000000000000CF
:1071C00000000000000000000000000000000000BF
:1071D00000000000000000000000000000000000AF
:1071E000000000000000000000000000000000009F
:1071F000000000000000000000000000000000008F
:1072000010B5054C237833B9044B13B10448AFF3E0
:1072100000800123237010BDB82100200000000071
:10722000D423030008B5034B1BB103490348AFF354
:10723000008008BD00000000BC210020D423030012
:10724000154B002B08BF134B9D46A3F5803A002138
:107250008B460F461348144A121A09F0C7FF0F4B0A
:10726000002B00D098470E4B002B00D098470020F1
:10727000002104000D000D48002802D00C48AFF397
:10728000008009F055FF2000290006F027F809F0DA
:107290003BFF00BF000008000000042000000000C9
:1072A00000000000B82100204C5800200000000021
:1072B000000000000649074A074B9B1A03DD043B08
:1072C000C858D050FBDC00F063FFFFF7B9FF0000A7
:1072D000CC240300681F0020B8210020FEE7FEE751
:1072E000FEE7FEE7FEE7FEE7FEE7FEE7FEE7FEE776
:1072F000F0B595B0002415460F4608461E4603F02B
:1073000083FE384623460895082205A91A9D09964A
:107310000D950A948DF82C400C9403F0CFFE9DF847
:1073200014308DF81140DDE9061003F00302012A44
:10733000CDE9020127D0022A04D0384603F068FEC6
:1073400015B0F0BDBDF81650C3F3C2038DF8103070
:10735000AD090826082D2C4628BF082433462246AE
:107360000EA9384603F0AAFE2D1B214608AB02AA3F
:107370000EA8264400F05CFE002DEBD1384603F049
:1073800047FE15B0F0BDBDF81460059DC6F3831629
:10739000C3F3C204B2000EA9384608238DF810408A
:1073A000C5F3952503F08AFE08AB324628460EA9A0
:1073B000009302AB00F096FD384603F029FE15B0AD
:1073C000F0BD00BF014B01221A7070471822002047
:1073D000704700BF00B583B0044B0093044A4023BC
:1073E000FFF786FF03B05DF804FB00BFF5730200F2
:1073F000D821002038B50E480E4D03780E4CEB5CBA
:107400000025D2B2257053B90C3004F07FFF58B973
:107410000A4B1B7813B12378002BFCD038BD043005
:1074200005F02AFA0028F3D001F090F9F0E700BF48
:10743000681F00203058002018220020D42100208E
:1074400070B51348134A0378D35C88B0DBB90C30AD
:1074500004F0DEFE104D0FCD6C460FC495E80F0012
:1074600008AD142645F8206D84E80F002946002257
:10747000074803F09DFF08B101F068F9074B0022AF
:107480001A7008B070BD043005F05CF9E2E700BF87
:10749000681F00203058002044120300D42100202F
:1074A00070B50D4D0FCD88B06C460FC495E80F0038
:1074B00008AD142645F8206D84E80F002946074AD8
:1074C000074803F075FF08B101F040F9054B0122B0
:1074D0001A7008B070BD00BF44120300C5730200EB
:1074E000681F0020D421002008B5FFF7D9FF042130
:1074F000034800F0ADFC034B01225A7108BD00BFE8
:10750000B42403007C1F0020F0B5324C85B004F594
:10751000836002F0A5FC04F2144002F0A1FCD4E95F
:10752000013703EA0702D01C04EB800114F82000A5
:1075300010F0040044D003F1020C0E7806F00306AC
:10754000012E654635D0022E02F1030621D004EB50
:1075500086010028F1D104EB82020133D268019246
:107560003B4004EB830302F00302012ADE6829D0CA
:10757000022A23D1BDF806309B090333360C05EBF4
:107580009305154802F078FC00B16560304605B0FF
:10759000F0BD4B880CEB931307EA0302D11C03F1F7
:1075A000020C14F82100654604EB810100F0040090
:1075B000CFE70B88C3F383136344EDE70026E0E7CE
:1075C0009D1CC8E7BDF80430C3F38313360C1D447B
:1075D000D7E700BFEC220020002700200B4B0C480F
:1075E00010B50022FF21C3F818249960C3E90022D6
:1075F000C3F8142483F8202403F0C2FC044610B915
:10760000044803F08FFD204610BD00BFEC2200208F
:10761000102403008412030021B9124B03EBC000B5
:1076200000687047104A0F49521AD20815D030B47A
:107630000E4D2B88834212D0002303E035F82340FF
:10764000844205D001339A42F8D1002030BC704703
:1076500001EBC300006830BC704710467047084615
:10766000F8E700BF24240300AC240300B421002069
:10767000094B013903EBC00003290BD8DFE801F007
:10768000020806040220704740797047007970476D
:107690000420704700207047242403002DE9F043A4
:1076A00083B002AB002203F8012DDFF8DC9007461F
:1076B00018468846D9F8084001F0D4FBD9E90132D0
:1076C000D9F80060134401339B1B012B58D809F2F1
:1076D0001C450121284602F0ABFBFFF715FF0146D0
:1076E000284602F0A5FBD9E90132D9F8001013446D
:1076F00001335B1A012BECD90A4003320523023116
:107700009DF8070049F82230C9F8001001F0D0FBBD
:1077100000211C4802F082FB80F31000731C234000
:1077200009EB830300043440033440EA1740D86077
:1077300019F8243067F3C50309F8243039F82430E8
:107740006FF3891329F8243059F8242068F39F2215
:107750001346012161F301036FF3820349F82420EA
:1077600009F8243099F820341BB906E000F00EF82F
:1077700018B1D9E900329A42F8D103B0BDE8F083DC
:107780003146B9E708270020EC2200202DE9F04718
:10779000934C002384B0C4F81834BFF34F8FD4E95E
:1077A000015605EA0602D31C04EB830114F82330CA
:1077B000580719D527680B7803F00303012B43D032
:1077C000022B03D14B88023505EB931506EA05021F
:1077D000D4F81804D31C04EB830128B9AF4239D97B
:1077E00014F823305B07E6D404EB82026B1CD268EA
:1077F0000192334004EB830302F00302DB6802933F
:10780000022A05F1020700F08D80012A26D0D4F863
:1078100010543DB12B6828469B689847EB681D685B
:10782000002DF7D16F48704B7049C01AC008000492
:1078300040F00200FFF732FFD4E90030C01A18BF51
:10784000012004B0BDE8F0870B880235C3F3831331
:107850001D44BBE7676004B0BDE8F087BDF80420B5
:107860006348C2F38313062B28BF062363F38912F0
:1078700002339900ADF8042003F084FB8046002811
:10788000C5D003F0C1FB0023082201A9404603F044
:10789000E1FBBDF8043013F4707F00F09F806FF0BF
:1078A000010AAAEB050A082506EA070103312B465F
:1078B000042204EB8101404603F0CCFBBDF8043008
:1078C00007F101090AEB0902C3F3831393424F4600
:1078D00005F10405E8D8D4F81834002B68D1D4F8A1
:1078E000105465B1EB685A7928464146002A5BD0AE
:1078F0002B681B689847EB681D68002DF2D1404645
:1079000003F086FB04A8002300F80D3D01F0AAFA5D
:10791000D4F818340BB9C4F804909DF8030001F0B2
:10792000C7FA89E7BDF8063031484FEA93194D464A
:10793000502D28BF502565F38F1305F10801ADF8D0
:10794000063003F01FFB804600283FF460AF26EAB4
:10795000070A0AF1010A03F057FB4FEA8A0A0023DB
:10796000082201A9404603F075FB55452BD9EBB21F
:10797000BAF1000F20D006EA0701A3EB0A03033196
:1079800004EB8101DDB252460823404603F062FB5E
:107990002A460AF108031749404603F05BFB09F148
:1079A000030907EB990996E71D68002D9AD1A6E710
:1079B000404603F02DFB3FE72A4608230D49404689
:1079C00003F048FBEBE706EA0701033104EB810112
:1079D0002A460823404603F03DFBE0E7B9467AE734
:1079E000EC2200204C240300242403009012030006
:1079F00010240300F82200202DE9F04782B002ABEA
:107A0000002403F8014DDFF8ECA007461846914624
:107A10008846DAF8084001F025FADAE90132DAF8A6
:107A20000060134401339B1B022B5ED80AF21C45F5
:107A30000121284602F0FCF9FFF766FD01462846C1
:107A400002F0F6F9DAE90132DAF8001013440133F2
:107A50005B1A022BECD90A400332033145239DF80F
:107A600007004AF82230CAF8001001F021FAB31CCE
:107A700023400AEB830300211D48C3F80C9002F059
:107A8000CDF980F31000731C23400AEB830300043C
:107A90003440033440EA1740D8601AF8243067F3C2
:107AA000C5030AF824303AF82430012161F3891320
:107AB0002AF824305AF8242068F39F22134661F3F1
:107AC00001036FF382034AF824200AF824309AF85D
:107AD00020341BB906E0FFF759FE18B1DAE900328D
:107AE0009A42F8D102B0BDE8F0873146B3E700BF53
:107AF00008270020EC2200202DE9F04F83B002ADD2
:107B0000002405F8014D3B4C8046284693469A4692
:107B10008946A56801F0A6F9D4E901322768134423
:107B20000133DB1B032B63D804F21C4601213046D2
:107B300002F07EF9FFF7E8FC0146304602F078F9E2
:107B4000D4E901322168134401335B1A032BEDD9C8
:107B50000A400332852344F8223004319DF807009F
:107B6000216001F0A5F9BA1CFB1C2A402B4004EB54
:107B7000820204EB830300211F48C2F80CB0C3F853
:107B80000CA002F04BF980F310007B1C2B4004EB9F
:107B9000830300043D40033540EA1840D86014F8E0
:107BA000253068F3C50304F8253034F82530022267
:107BB00062F3891324F8253054F8252069F39F22B5
:107BC0001346012161F301036FF3820344F825207A
:107BD00004F8253094F820341BB906E0FFF7D6FDF1
:107BE00018B1D4E900329A42F8D103B0BDE8F08F61
:107BF0003946ADE7EC220020082700202DE9F04FA0
:107C000083B002AE002406F8014D3E4C804630465B
:107C100093469A46A568894601F024F9D4E90132D1
:107C2000276813440133DB1B042B69D804F21C467C
:107C30000121304602F0FCF8FFF766FC01463046B1
:107C400002F0F6F8D4E901322168134401335B1ADB
:107C5000042BEDD90A400332C52344F82230053104
:107C60009DF80700216001F023F9B81CFA1C284098
:107C70002A403B1D2B4004EB800004EB820204EB06
:107C80008303C0F80CB00021C2F80CA01E480C9A67
:107C9000DA6002F0C3F880F310007B1C2B4004EB89
:107CA000830300043D40033540EA1840D86014F8CF
:107CB000253068F3C50304F8253034F82530032255
:107CC00062F3891324F8253054F8252069F39F22A4
:107CD0001346012161F301036FF3820344F8252069
:107CE00004F8253094F820341BB906E0FFF74EFD68
:107CF00018B1D4E900329A42F8D103B0BDE8F08F50
:107D00003946A7E7EC220020082700202DE9F04F94
:107D100087B006AE002406F8114D454C109F04971D
:107D2000CDE90223804699463046119B0593924641
:107D3000A5688B4601F096F8D4E901322768134410
:107D40000133DB1B052B70D804F21C4601213046A1
:107D500002F06EF8FFF7D8FB0146304602F068F8F3
:107D6000D4E901322168134401335B1A052BEDD9A4
:107D70000A40033240F2051344F8223006319DF8E0
:107D800007002160FE1C01F093F8B91C29402E4029
:107D90003A1D2A4004EB810104EB86067B1D2B4033
:107DA00004EB8202C1F80CA004EB8303C6F80C902C
:107DB000109ED6600021119A1E48DA6002F02EF85B
:107DC00080F310007B1C2B4004EB830300043D4038
:107DD000033540EA1840D86014F8253068F3C5032D
:107DE00004F8253034F82530042262F3891324F88E
:107DF000253054F825206BF39F221346012161F3AF
:107E000001036FF3820344F8252004F8253094F829
:107E100020341BB906E0FFF7B9FC18B1D4E90032F1
:107E20009A42F8D107B0BDE8F08F3946A0E700BF0D
:107E3000EC22002008270020044BD3E900239A42BB
:107E400001D0FFF7A3BC0020704700BFEC22002048
:107E500030B4184DD5F8104400215CB1E3681A79AC
:107E60008A4204D116E0DB681A798A4212D01B6874
:107E7000002BF8D1C3681971D5F8103493B1DA68C2
:107E8000C36812681A60D5F81034DB68186030BC1B
:107E90000846704701310A29DFD14FF0FF3108460B
:107EA00030BC7047C5F81004C2681360084630BC87
:107EB000704700BFEC22002038B5094BD3F81044BE
:107EC000012583F820544CB1E3685D712368204696
:107ED0005B689847E3681C68002CF5D138BD00BF8B
:107EE000EC2200202DE9F04784B01D460C9C0023B5
:107EF00094F80C802373EB8881460E461746002BBE
:107F000040D1297A05290ED06B7AA88873BB404BE3
:107F100053F821A00021FFF77FFB524603463D495D
:107F2000204602F021F8062F09D8DFE807F0046A9E
:107F30004249525D33004946204602F015F82B7A3B
:107F4000052B05D06B7A5BB93349204602F00CF85B
:107F5000204601F0FDFF84F80C8004B0BDE8F087F6
:107F60002E4A2F49204601F0FFFFEDE7FFF780FB87
:107F70002C4B2B4953F82020204601F0F5FF297A9D
:107F8000A888C4E7254A00922749284A204601F0DC
:107F9000EBFFB6E7D6E90410D6E900230390D6E953
:107FA00002070291CDE900074946204601F0DCFFB7
:107FB000C5E74946D6E90023204601F0D5FFBEE7D4
:107FC000B168D6E9002320460091494601F0CCFF74
:107FD000B5E7D6E90201D6E90023019100904946B0
:107FE000204601F0C1FFAAE7D6E90371B068D6E9DF
:107FF00000230291CDE900074946204601F0B4FF75
:108000009DE732684946204601F0AEFF97E700BF82
:108010001C1303000C1303001813030000130300C8
:1080200008130300A8120300E8120300E012030083
:10803000082900D970472DE9F04F1D4690460023CE
:108040002A7B2B7385B0B8F80630039207460E469C
:10805000002B7BD198F80810052911D098F8093029
:10806000B8F80400002B63D13C4B53F821400021A9
:10807000FFF7D2FA224603463949284601F074FF39
:10808000DFF8FCB0DFF8FC90002405E03A5D013435
:1080900001F06AFF082C09D0A64249462846F5D8C7
:1080A0005946013401F060FF082CF5D12D49DFF865
:1080B000D8B0DFF8D890284601F056FF00240CE035
:1080C00017F804A0BAF17E0F23D92E22494628467C
:1080D000013401F049FF082C08D0A642F0D85946D7
:1080E0002846013401F040FF082CF6D198F80830FA
:1080F000052B02D098F80930A3B91B49284601F096
:1081000033FF284601F024FF039B2B7305B0BDE825
:10811000F08F09F031F850445246437813F0970F2E
:10812000D3D0D3E7114A1249284601F01DFFE4E7F6
:10813000FFF79EFA0F4B0E4953F82020284601F016
:1081400013FF98F80810B8F804008DE7074A00926A
:1081500009490A4A284601F007FF7BE71C13030080
:108160000C130300D81203001813030000130300BC
:1081700008130300A8120300E8120300E012030032
:10818000D4120300CC12030014130300DC1203000A
:1081900010B44FF080414FF080520020C1F80C0124
:1081A0005E4BC1F81001C1F83805D2F80414C3F8C9
:1081B0002015D2F80814C3F82415D2F80C14C3F80B
:1081C0002815D2F81014C3F82C15D2F81414C3F8DB
:1081D0003015D2F81814C3F83415D2F81C14C3F8AB
:1081E0004015D2F82014C3F84415D2F82414C3F86B
:1081F0004815D2F82814C3F84C15D2F82C14C3F83B
:108200005015D2F83014C3F85415D2F83414C3F80A
:108210006015D2F83814C3F86415D2F83C04C3F8DA
:108220006805D2F840043E49C3F86C050968D2F8E5
:108230004424C3F87025082924D04FF08043D3F894
:108240000024D20744BF6FF00102C3F80024354A6E
:10825000D2F8883043F47003C2F88830BFF34F8FF0
:10826000BFF36F8F4FF01023D3F80022002A23DBD7
:10827000D3F80432002B1FDB2B4B2C4A1A605DF81D
:10828000044B70472A4B1B68002BD6D129482A4A39
:108290002A4C04602A492B4BFB20C2F818050A68B7
:1082A0001B68294822F00F0203F00F0313434FF419
:1082B00000720B600260C0E7244B0122C3F8042562
:1082C000D3F80024002AFBD04FF0102312221F49BC
:1082D000C3F80022D1F80034002BFBD04FF010225D
:1082E00012211A4BC2F80412D3F80024002AFBD042
:1082F00000221649C3F80425D1F80034002BFBD026
:10830000BFF34F8F0749124BCA6802F4E062134370
:10831000CB60BFF34F8F00BFFDE700BF00C0004040
:108320003001001000ED00E0841F00200090D00319
:10833000340100108C56004000F0004048810300DA
:10834000E40E0040580200104096024000E0014058
:108350000400FA0570B51A4B1D789DB1194B1C68C5
:108360002378C0B2984210D004F10802002306E03E
:1083700014F833108142164602F1080206D0013388
:108380009D42F5D100231B78FFDE264603F072FAEA
:108390007378A3F10103B3FA83F35B09834200D03E
:1083A00070BD094BD3E900231343F9D1074B0848AB
:1083B000196800224908BDE8704000F003BD00BF05
:1083C000A8270020F8270020D0270020AC27002075
:1083D000B02700202DE9F04F9D4E337887B0002B59
:1083E00000F030819B4F9C4DDFF8788200244FF0E5
:1083F0000109D7F800B01BF8340003F03BFA0BEB8F
:10840000C4031BF834B05B784FEA5B0C1BF0010E21
:1084100015F80C10A3F10103B3FA83F314BF0A0992
:1084200001F00F025B09042A00F2D080DFE812F0AD
:108430009800D000690048000500834200F0E98000
:10844000BEF1000F0CBFF0230F233078194005F860
:108450000C10A8B1D7F800C09CF800305B4500F0C4
:10846000E7800CF10802002304E01CF833105945A2
:1084700000F0DF8001338342964602F10802F4D116
:108480004FF000030DF117008DF817300023039310
:1084900000F0E8FCABF12002CBF1200329FA03F352
:1084A00009FA02F21A4309FA0BF103920291D8E990
:1084B0000023DDE9020122EA000023EA01017DE058
:1084C000834232780CD0BEF1000F0CBFF0230F2393
:1084D00003EA01030CBF04214021194305F80C10E5
:1084E0000134944285DBD8E90023134306D05B4B6B
:1084F0005B4819680022490800F064FC07B0BDE839
:10850000F08F834276D1BEF1000F14BF0F23F0230A
:1085100003EA0103327814BF30210321194305F81F
:108520000C10002ADFD0D7F800C09CF800305B4563
:1085300000F08B800CF108010023013393428E463A
:1085400001F10801CCD01CF833005845F5D1DEF814
:108550000430002BC4D05846012198473278BFE739
:10856000834233D1BEF1000F0CBFF0230F2303EA87
:1085700001030CBF0121102119434FF000030DF13D
:1085800017008DF817300023019305F80C1000F048
:1085900069FCABF1200309FA03F301930198CBF1D5
:1085A000200129FA01F1084309FA0BF10190009129
:1085B000D8E90023DDE900011043194302460B46C8
:1085C0009DF81700C8E9002300F072FC327887E7B5
:1085D000834213BF0023202302221A46BEF1000F5C
:1085E00012BF0F20F020134601400B4305F80C305A
:1085F000327875E7BEF1000F0CBFF0230F2303EABA
:1086000001030CBF01211021194305F80C10327829
:1086100066E7BEF1000F14BF0F23F02303EA010346
:1086200014BF30210321194305F80C10327857E7A5
:10863000E646DEF80430002B3FF422AF0021584616
:1086400098471DE7DFF81C804DE7E6467FE700BF4F
:10865000A8270020F8270020D8270020AC270020DA
:10866000B0270020D0270020092A40D9F0B583B0D8
:108670000E460546144602F087FF002831D0204AF6
:108680002049214B15600E70202200211F481C60DC
:1086900008F0ACFD1E4B00200021741EC3E9000150
:1086A000E4B236B305EBC4041A4E083D032701E0DB
:1086B000A5421ED09DF8063020788DF8047003F096
:1086C000FC036FF382038DF80630A3788DF8053034
:1086D000324601A902F062FF083C0028E8D003B04E
:1086E000F0BD02F007FF0028C9D003B0F0BD07209D
:1086F0007047094A0948002100F056FB03B0F0BD5D
:10870000F8270020A8270020AC270020D827002029
:10871000D027002055830200D58302008813030070
:1087200070B5084D2B785BB1074E002433680121EA
:1087300013F8340003F022F82B780134A342F5D863
:10874000002070BDA8270020F827002000B585B0C4
:1087500000230390194601AA44F20100CDE9013338
:1087600000F004F805B05DF804FB00BF10B572B668
:10877000FFF7A2FBFFF760FB0028FBD1104B114C69
:108780001149E41AE408240444F00100FEF786FFCE
:108790000E4B1B68DB0700D500BE44F002000C49FD
:1087A000FEF77CFFBFF34F8F0A490B4BCA6802F4F8
:1087B000E0621343CB60BFF34F8F00BFFDE700BF04
:1087C000242403004C24030098130300F0ED00E080
:1087D000A413030000ED00E00400FA05F0B412F069
:1087E000030412D14B1CDB000A4D0B4E0B4F3470AF
:1087F0009BB213442B600A4E0A4D0B4B28803A6003
:10880000347019802046F0BC704707242046F0BC25
:10881000704700BF00280020FC270020042800200B
:108820000C280020082800200A2800202DE9F04705
:108830002D4F3B888B4282B03CD3054602A84FF0B7
:10884000000800F8018D16460C4600F00BFB274B84
:10885000274A284819781378B0F800C09DF8070017
:10886000DBB2634538BF0133C9B238BF5FFA83F862
:10887000414523D092F800801378DFF88090DBB276
:108880009C4586BF0133DBB200235FFA88F8137082
:1088900000F00EFBD9F800300FFA88F24FEAC20A56
:1088A00043F83260534405B174B90020988002B097
:1088B000BDE8F087092002B0BDE8F08700F0F8FAC3
:1088C000042002B0BDE8F0870B4B38881B682946AE
:1088D00008FB0030224608F07EFCD9F800309A44AC
:1088E0000020AAF80440E2E7082800200C28002015
:1088F000FC2700200A28002000280020042800204F
:108900002DE9F84F1B4C1C4D22782B789A4226D02B
:10891000DFF86CA0DFF86C90184FDFF86CB04FF008
:1089200000082378DAF800203888D9F80060DBB234
:108930000FFA83FE02EBCE0103FB0060898852F838
:108940003E3098472378BBF80010DBB25A1C99429E
:10895000D2B206D9227023782A789A42E1D1BDE8B2
:10896000F88F84F8008022782B789A42D9D1BDE81C
:10897000F88F00BF0C280020FC27002008280020CA
:1089800004280020002800200A280020D0E9022323
:10899000D1E90201994208BF90422CBF012000207A
:1089A000704700BFD0E90030184700BF2DE9F04FF5
:1089B00087B0029000F0A0FB40B1AF49D1E900239D
:1089C00012F1807443F10005C1E9004500210298CD
:1089D000AA4E00F0ADFB002800F098803368002B11
:1089E00000F09480A64B34681B7823B11CB1237F20
:1089F000002B40F0538104AB039300230121029824
:108A0000336000F095FB002800F089809D489E4F60
:108A100000F0A0FB984BD3E90045D7E9002314EB05
:108A2000000845F10009994508BF90454046494670
:108A300003D218F1807049F10001DDF80C80C7E91C
:108A400000014146914801F0ABF900286FD1DFF8F1
:108A50004482DFF830A2DFF8209204E00D2800F015
:108A6000988000233360404602F09AFB3368002868
:108A700000F0F0806BB13368D0E90201D3E9022342
:108A8000994208BF90423ED233681B7F002B40F0D2
:108A9000C580404602F07EFB0746D7E902235046D8
:108AA000CDE9002300F056FBD9E90023764C12EB08
:108AB000000B43F1000CD4E900239C4508BF93450B
:108AC0005846614603D21BF180704CF10001DDE98C
:108AD0000023121A63EB01031946012A71F1000306
:108AE00053DB6B4DAA4200F29E80BA684FF49603A6
:108AF0000021504600F07AFA0028AFD13368002BED
:108B000000F0A180376007B0BDE8F08F04AB012111
:108B10000298039300F00CFB00287FF477AFDDF898
:108B20000C805A48414601F03BF900288FD0037869
:108B3000584D534F554C012B1FD079D3022B0ED1DA
:108B400028464FF0000902F025FB30B180F81C9058
:108B5000284602F01FFB0028F8D101233B70414654
:108B6000204601F04BF94146204601F019F9002852
:108B70003FF46DAF0378012BDFD141683368994230
:108B800065D0284602F010FBE9E70021504600F0CE
:108B9000C3FA3B4B1B78002B3FF463AF3B7F002BAA
:108BA0003FF45FAF504600F0D5FAD4E90023D9E98D
:108BB0000045241845F100059D4208BF9442204617
:108BC000294603D214F1807045F10001D7E9022350
:108BD000994208BF904246D33B69002B41D07B6944
:108BE0000493BB692C4A039805930821FFF71EFEE6
:108BF00000283DD1396900293FF433AF3B7F002B7A
:108C00003FF42FAFD7E90223541843F10005C7E919
:108C100002453946404602F0A9FA22E7316840464B
:108C200002F0A4FA35E7504600F094FA42195DE7E5
:108C300043681A7F002A92D101221A774168284698
:108C400002F094FA8BE7029800F0A2F95AE70023A9
:108C5000336084E7002B7FF456AF029800F09CF954
:108C600051E73B77BBE73946404602F07FFAF8E62A
:108C7000FFF76CFDBEE700BF1828002098280020F1
:108C800020280020881F0020902800207C28002019
:108C9000FFFFB400B8130300A5890200224800F0CA
:108CA00059FA224A224BD2E90089D3E9002318EB72
:108CB000000A49F1000B9B4508BF924550465946B2
:108CC00003D21AF180704BF10001D4E902239942DA
:108CD00008BF904223D3236903B9237763690493C0
:108CE00004A8A369134A039008210593FFF79EFD8A
:108CF00008B1FFF72BFD216900293FF47EAE237FE9
:108D0000002B3FF47AAED4E90223571843F1000850
:108D1000C4E902782146084802F028FA6DE62146A7
:108D2000054802F023FA66E6881F00201828002074
:108D300090280020A5890200B813030010B5134B3A
:108D400013491B68134882B058220193082300F08E
:108D5000D3FF044610B1204602B010BD0E4A0F48A2
:108D600001A900F0BDF804460028F4D101210B4808
:108D700000F0B8F901231946094A084800F010F933
:108D8000084B012220461A7002B010BDB413030034
:108D9000242800207C280020AD890200881F0020A4
:108DA000FFFF7F00202800204AB1A1F101010368E4
:108DB000B1FA81F14909C3E9041200207047072084
:108DC000704700BF037F0BB1002070472DE9F048CA
:108DD000826182B004461F480D4600F0BBF91E4B6D
:108DE0001E49D3E90023D1E9006712EB000B43F1E0
:108DF000000CBC4508BFB34503D21BF1807B4CF18E
:108E0000000C1BEB050221694CF10003C4E90223AD
:108E100079B901A9124800F087FF88B100254460A4
:108E2000057001A90E4800F0ABFF68B902B0BDE8BB
:108E3000F088256101A90A4800F076FF0028EDD1ED
:108E4000042002B0BDE8F088024800F087F9284607
:108E5000ECE700BF881F0020182800209028002081
:108E60007C28002070B4EFF3108472B60D4B9A6822
:108E7000AAB90D490D4E01259D60D1F880503540AD
:108E80001D60C1F88060D1F884505D604FF0FF3301
:108E9000C1F88430027004B962B670BC7047012317
:108EA0000370F8E72458002000E100E0FC06FFBD55
:108EB000094B9A687AB170B910B4EFF3108172B6A9
:108EC000064A1C6814605C685460986001B962B618
:108ED0005DF8044B704770472458002000E100E023
:108EE000F8B5234E4579234C234F0346234847F8D2
:108EF0002520801B04EBC506C0083679000486BB1C
:108F00001A680D88C2F8085593F904208978002A58
:108F10001FDB02F1604202F561424901C9B282F8E9
:108F2000001393F90420164F1649012602F01F057D
:108F3000520906FA05F547F822505A7904EBC205A2
:108F400040F003002E7144F83230FEF7A7FB0020FA
:108F5000F8BD0D4D02F00F0249011544C9B2297642
:108F6000DFE740F002000949FEF798FB0820F8BD52
:108F7000242403009C280020A42800205C24030053
:108F800000E100E0FC130300FCEC00E0D813030058
:108F9000036801221A607047036801225A60704713
:108FA000F0B404684FF480358D40C4F80853066867
:108FB0008C00C6F8485304F5A0740668A4B20027D4
:108FC000375182B036590468019601F5A87122F034
:108FD0007F42019E44F821200268C2F8445313B135
:108FE0000368C3F8045302B0F0BC70472DE9F047A2
:108FF00088464FF48037016807FA08F7C1F84873CC
:109000000168C1F80873064600684FEA8804011930
:10901000D0F80455D1F84005C1F8405504F5A074C6
:10902000A4B231684FF0000941F8049082B0401BAF
:109030000959009120F07F4001289A4622F07F458F
:10904000009B0BD1264B4FF4806043F001039847FF
:10905000336843F804901B590193019B3368D3F89C
:109060000445C3F844732B1B23F07F43012B08F501
:10907000A87817D130681A4B013540F8285043F0D2
:1090800001034FF4806098473268D2F804359C425F
:1090900022D1C2F8447333680020C3F8047302B0CD
:1090A000BDE8F087336843F828503268D2F80415D9
:1090B0006B1ACAF1FF1A013B0AF57F4A23F07F437E
:1090C0009A4509D3002BE4D1013542F82850326883
:1090D000D2F804359942DCD00D2002B0BDE8F0870B
:1090E000D013030002680223C2F8443311B10268AE
:1090F000C2F80433704700BF0368D3F8040150B1CD
:10910000002282B0C3F80421D3F804310193019BFB
:10911000012002B0704770474FF48033026803FAB1
:1091200001F1C2F848130368C3F80813704700BF81
:10913000890001F5A07189B20368585840B1002236
:109140005A5082B05B580193019B012002B07047D6
:10915000704700BF0368D3F80405704790F90430E6
:1091600005485A09403203F01F03012101FA03F3B5
:1091700040F82230704700BF00E100E0024A034B94
:1091800010681B68184700BF9C280020A4280020F6
:10919000F0B5344D344EB5F802C06A684FEA8C071A
:1091A00007EB0C0306EB830383B0596801F5805489
:1091B000002A53D05388033302EB8302944231D9FF
:1091C000136801332ED05388033302EB8303A34289
:1091D00028D84FF6FF7E9088704517D01088A8B128
:1091E0009068013012D06A605388204C2048A688CD
:1091F0002168033300249BB200949B0001EB86019D
:1092000003242C7001F0D6FA03B0F0BD9C4209D9BA
:109210001A6801321A4605D05888033003EB8003E0
:109220009C42D8D2674406EB8706F3686BB10F4BBC
:109230000F48196802229A800524002301222C700D
:1092400003B0BDE8F04001F053BB094804240122FB
:109250002C7003B0BDE8F04001F04ABB01F10802F8
:10926000ACE700BFCC280020E42800202029002003
:10927000A0210020F0B443681BB1394AD468A3424E
:1092800049D20023374F0B807A684FF0010C02F56A
:1092900080554FF6FF76083295420ED8BCF1020F8A
:1092A000A1F800C007F1140757D07A6802F580557D
:1092B000083295424FF0020CF0D913680133EDD01B
:1092C0005388033302EB83039D42E7D39488B4426F
:1092D0000DD014885CB19468B4F1FF3F07D00368E7
:1092E000A34211D05388033302EB8302D4E79D429B
:1092F000D4D91A6801321A46D0D05C88033403EB03
:1093000084039D42E2D2C9E7174B42601B89038167
:109310000120F0BC704712699342B2D813F00305E4
:10932000AFD1114A048912899442AAD104689A687B
:109330009442A6D10B484268934203D902F5805269
:10934000934207D38269934207D902F58052934230
:1093500003D201250D800120DBE70020F0BC70471F
:10936000A0210020E4280020CC2800202DE9F04F87
:109370009F4F8BB004464FF6FF783E68002E00F0FA
:10938000C2803278531E052B00F2B680DFE803F06E
:10939000593B3B1E1E03002C40F0BC80DFF874C21A
:1093A0009CF80C209CF80030002A00F05981013B09
:1093B0008CF80C40062B00F29F80DFE813F0AD0321
:1093C000BC02B801DB019D00CE02BF02002C40F0C0
:1093D000A1803379012B00F07781C0F04E8105AD7B
:1093E000022B0594C5E902442C6100F09C8048F2F0
:1093F0000E6006903378023B042B33D8DFE803F08D
:1094000058684C2C6400B6F81490B17D002C40F0E4
:1094100007814FEA8904774D04EB090305EB8303C9
:10942000B3F808A05B6803EB8A0A062900F21C83E4
:10943000DFE811F04002B801D801EB01FF011A0288
:109440003302002C40F0C8803379032B00F28E8069
:10945000DFE803F0B6A2976B04238DF81430F3888D
:10946000ADF82030644C04F1100654F8043B284653
:1094700003B19847A642F8D16049614800243C6096
:1094800000F0BCFC01215F4800F0DEFC00287FF406
:1094900074AF0BB0BDE8F08F03238DF81430F38860
:1094A000ADF820303389ADF82230F3680793D9E75F
:1094B00001238DF814303389ADF82030B388ADF82E
:1094C0002230F3680793CDE705238DF81430C9E700
:1094D00002238DF814303389ADF82030B388ADF80D
:1094E0002230F3680793B37DA3F10603B3FA83F345
:1094F0005B098DF82430B5E705AD0023AB6005931B
:10950000C5E9033373E73D493D4800F049FC064691
:10951000386036E705AD0023AB600593C5E903333A
:109520004FF4064065E7204663E7374C374A216829
:109530003748304D4FF0000986F804900823CDF8E5
:10954000009001F037F9334B26685B88A18803EB64
:10955000830305EB830205F82390536823600223FD
:1095600056601181A380002893D03E682A4A05AD39
:10957000002353600593C5E902332B6148F20D6067
:1095800037E7214A2248116800230224337194806E
:10959000012201F0ADF9E6E7164D2B78022B00F021
:1095A000DA822B7D022B00F0BA821B4B05AD002026
:1095B00001221A7005905860C5E90200286118E779
:1095C000114B164A19681248012333710023009386
:1095D000082301F0EFF8C6E705AD0F4A00235360FA
:1095E0000593C5E902332B614FF4064001E700BF44
:1095F000E0280020E4280020B4280020DC280020F7
:109600000C2900201C29002020290020141403000C
:10961000A0210020CC280020C42800201C14030016
:109620000229F2887FD94FEA8904B54D04EB09017C
:1096300005EB8101D31C0A8913440B81F28804EBEA
:10964000090105EB810105AD4B89033B9B1A002203
:109650004B81AA600592C5E903224FF40640C8E693
:10966000072B00F2EB81DFE813F0B201E901E90119
:109670005B019F01690169018B0102233371CDE90F
:10968000064405ADF368059328460DF11201FFF776
:10969000F1FD002800F02A8106999A4A8B88F38010
:1096A0000B883381984800940423BDF8124001F0E0
:1096B00081F8002840F04382914B04EB840403EBD3
:1096C000840401232374E4E6904B1B78002B00F004
:1096D000FF80DFF83CE2BEF80490B9F1010F15D825
:1096E000874D039409EB890205EB8202043212F8DC
:1096F000043C002B00F0BC8109F1010399B201295F
:109700009946AEF8043002F11402F0D905AD0822F2
:1097100000217F4807F06AFD0020A8600590C5E998
:1097200003003E6865E6764D4FEA890487E779488D
:10973000DCF804208488016853887348033301EB04
:109740008401002400949BB203249B008CF8004009
:1097500001F030F800283FF49CAE05AD002341F63F
:109760001D523E68AB600593C5E90333904208BFC4
:1097700018463EE6BCF80230614D03EB830305EB6F
:109780008305EB68002B00F0BC81624B5E481968D2
:1097900002229A8005228CF800200023012201F089
:1097A000A7F8D7E7032A0CBF052306230022B375C9
:1097B0000AF104010092042306F10802524800F065
:1097C000F9FF00283FF465AEB37DF288022B48F222
:1097D0000D6065D8A14405EB89056B89033B9B1A95
:1097E0006B81BAE733694848002B14BF0323012378
:1097F0000022B3750AF108010092042306F10C025D
:1098000000F0D8FF0028DFD143E6F38832693E48F4
:109810004FF0010C86F816C04FF0000C0AF10C0155
:109820009B00CDF800C000F0C5FF00283FF431AE2A
:10983000CAE7394BB26939491A604FF0000B184634
:10984000C3F804B0FFF716FD002800F07C81022366
:10985000B37504235146CDF800B0F2182A4800F041
:10986000A9FF0028B0D114E62C4B2B4AB3F800A076
:1098700051682548234A00234FF0060C86F816C08D
:109880000093042300F096FF00289DD10AEB8A0A7A
:1098900005EB8A0501232B74FBE5F28841F61D5088
:1098A00004EB090105EB8101D31C0A8913440B81E8
:1098B000F2888FE702230022B375042300925146F9
:1098C000F218114800F076FF00283FF4E2AD7BE784
:1098D00005AD082221460E4807F088FC0594C5E92D
:1098E00002442C613E6848F2016082E548F209605A
:1098F0000023C5E90033C5E902332B6179E500BFD8
:10990000E428002010140300A0210020C428002017
:109910002C29002020290020A82800202829002008
:10992000904ADCF804109388498803330B440221E1
:1099300093808CF80010FFF72BFC0BE7894B8A4AC9
:1099400019688A4800230093CCF8043007238CF868
:109950000030082300F02EFFFCE6BCF80220844D06
:109960009300134405EB8305062000236968814AB0
:1099700000938CF8000008237C4800F01BFFE9E608
:1099800001238CF800309CF80A30002B3AD0784D37
:10999000EB6800228CF80A20A3BB2A7C92B3ACF8B7
:1099A0000230FFF7F5FBD5E6BCF80220704D6D4C98
:1099B0009300991805EB810120684E68B4F804E023
:1099C000486002202660A1F808E0A080C9E7684D41
:1099D000BCF808102A7D2B78B2FA82F252090131C4
:1099E000B3FA83F35B098CF80B20ACF80810002263
:1099F00001218CF80A30ACF802208CF80C208CF88D
:109A00000010C2E79CF80B3053B1594D2B6A00226D
:109A10008CF80B2023B995F824300BB10123BEE755
:109A200005AD0020A8608CF80000ACF80200CCF86E
:109A300004000590C5E903003E68DAE4013B062B0B
:109A40003FF65AAD01A252F823F000BF199B020065
:109A5000379902002F97020075970200F9940200CF
:109A60005B9902003D990200F28848F20E6017E708
:109A70001368DEF8001003F5805C03F1080A002982
:109A800048D04B88033301EB83018C4503D8039BFB
:109A9000CEF8003030E60B680133F8D04B88033342
:109AA00001EB83039C45F2D3888840451CD0B1F874
:109AB00000B0BBF1000F17D08C68013414D0F388CC
:109AC000CEF800108342DAD1002300932A4A2748B7
:109AD000042300F06FFE00283FD109EB890905EB54
:109AE000890501232B74D4E49C45D0D91968013130
:109AF0001946CCD05888033003EB80039C45D3D261
:109B0000C5E704228CF8002069681848012200F09B
:109B1000EFFE1FE65146B8E79CF80A3035E701230F
:109B20009A001A4405EB820300205968009008232C
:109B300005F822000F4A0D4800F03CFE13E53E6890
:109B400048F20D60D4E605AD0590C5E90200286134
:109B500048F209604DE40023E2E73E6848F20D60F8
:109B600005ADC5E6202900201C140300A02100201B
:109B7000E428002014140300101403004068FFF7C9
:109B8000F5BB00BF054A064913686FEA93336FEAD5
:109B900083330120087013600020704734290020AF
:109BA00038300020204B1B7833B310B309B30B6857
:109BB0005A1EFF2A31D8202BF0B414D80024234693
:109BC0001A4F3E68082B26FA03F234BF20254FF4C3
:109BD0008075D20713D401330E2B2C44F2D148F2F6
:109BE0000410F0BC7047402B1AD94FF4807408233E
:109BF000E6E748F20E10704748F2081070474FF041
:109C0000010C0B4A0CFA03F326EA03061444046021
:109C10003E6000200D60F0BC704748F207107047AE
:109C2000202BCBD9E1E700BF3830002034290020B9
:109C3000382900202D4B1B78BBB3B0B32C4B984276
:109C40003ED003F1200290423CD003F1400290420A
:109C50003AD003F16002904238D003F18002904282
:109C600036D003F1A002904234D003F1C0029042FA
:109C700032D0E033984231D0203398421ED003F5E1
:109C8000807290422CD003F5007290422AD003F5E6
:109C90004072904228D003F58062904206D003F5CE
:109CA000A063984208BF0D2001D070470C201149D5
:109CB00001220B68824013430B6070470820F6E7CF
:109CC0000020F4E70120F2E70220F0E70320EEE7AE
:109CD0000420ECE70520EAE70620E8E70720E6E7AE
:109CE0000920E4E70A20E2E70B20E0E73830002013
:109CF000382900203429002099B110B4B2FBF3F4C4
:109D000003FB1424A4B244B9C0E900148460828126
:109D1000C38120465DF8044B704709205DF8044B71
:109D200070470E20704700BF30B482B050E8013F4A
:109D30009DB2C48925448489A54228BF2D1B04896E
:109D4000A54202BFBFF32F8F002207E0C5EA03053B
:109D500040E80154002CE9D14FF001028DF80320B6
:109D60000193019B9DF803200B602AB10B880068CA
:109D7000184402B030BC704702F0FF031846F8E701
:109D80000A884B889A4201D00020704750E8012F82
:109D9000C2EA024240E80123002BF7D101207047BC
:109DA00030B482B050E8023F1FFAA3F5C488A54240
:109DB00002BFBFF32F8F00220DE0C48925448489A0
:109DC000A54228BF2D1BC3EA054540E80254002CDC
:109DD000E8D14FF001028DF803200193019B9DF81B
:109DE00003200B602AB14B880068184402B030BCD5
:109DF000704702F0FF031846F8E700BF0A884B8857
:109E00009A4201D00020704750E8022FC2EA224255
:109E100040E80223002BF7D10120704750E8002FC3
:109E20000B4640E8003C9CF0000FF7D1104670470D
:109E300050E8003F03EB010240E8002C9CF0000FCB
:109E4000F6D11046704700BF50E8003FA3EB010277
:109E500040E8002C9CF0000FF6D11046704700BF80
:109E6000012350E8002F42EA030C40E800C191F0C2
:109E7000000FF6D160467047002350E800CF0CEA8F
:109E8000030240E8002191F0000FF6D160467047D0
:109E9000B8B130B4D0E90112521A0468D2B2531EDC
:109EA0002160DBB242B101680A685C1E551C0D607E
:109EB0001370E3B2FF2BF6D103680020187130BC99
:109EC00070470E20704700BFF0B583B002AB00258D
:109ED00003F8015D04461846FEF7C4FFD4E90031DB
:109EE0001A688A4210D9511E19602168A3680F6848
:109EF00012F8015C0A79268AE068DB1BDBB29A4221
:109F000006FB050538BF0B719DF80700FEF7D0FF73
:109F1000284603B0F0BD00BF30B583B002AB0022CD
:109F200003F8012D054618460C46FEF79BFF2A68EC
:109F30001368591C1160E9682A8A641AB4FBF2F4A8
:109F40001C709DF80700FEF7B3FF03B030BD00BFE3
:109F5000826842B110B504464369016800699847B8
:109F60000023A36010BD70470EB400B582B0039902
:109F700029B102AA04AB42F8043D00F0A9F802B0EE
:109F80005DF804EB03B070472DE9F04F924683B0C3
:109F900051450F4605461E46DDE90CB2C0F09280E1
:109FA0000B464FF00108B3FBFAF39A4508F101089C
:109FB000F9D9B04538BFB04612F00109A96802D1FD
:109FC000BBF1000F54D1012402E0013E0AFB04F46E
:109FD000012EFAD8B7FBF4F08245F7D93B4E02E0E8
:109FE000A968B7FBF4F0335C2A680A2B04FB1077EE
:109FF00002EB010E01F1010029D0A8608EF80030BB
:10A00000D5E90131994202D32846FFF7A1FFB4FBFD
:10A01000FAF4002CE4D1B9F1000F15D0BBF1000F18
:10A0200012D0C34510D92024AB682A68591CA960F6
:10A03000D454D5E901329A420BF1FF3B14D2BBF163
:10A04000000F01D0C345EFD103B0BDE8F08FA86089
:10A050004FF00D005054D5E9011088421DD22968F7
:10A0600001EB000E0130C8E72846FFF771FFE6E775
:10A07000930722D42024C345A5D92B684A1CAA6083
:10A080005C54D5E9013199420BF1FF3B10D2BBF191
:10A09000000F98D0C345F0D195E728460193FFF70C
:10A0A00057FFAA682968019B501C01EB020EA4E728
:10A0B0002846FFF74DFFA968E9E7002E0CBF3024C2
:10A0C0002024D8E74FF0010873E700BF30140300E5
:10A0D000002900F0B9822DE9F04F054687B091467E
:10A0E0000C460E78DFF8C8A64FF00D0B13E0AB68F6
:10A0F00028680A2E03F1010200EB030100F04B82F5
:10A10000AA600E70D5E901329A4280F01B81267850
:10A11000002E00F01E810134002E00F01A81252E41
:10A12000E5D12346002713F8012B2D2A00F0E38008
:10A13000302A00F0E4802B2A00F0D4802A2A00F094
:10A140000D81A2F13006F1B2092903D97DE2A1F116
:10A1500030060346184606EB860110F8012BA2F1E3
:10A160003004092C02EB4101F1D92E2A00F00281C2
:10A170004FF00008013301E013F8012B02F0FB015E
:10A1800068291C46F8D0253A532AC0D801A353F8B1
:10A1900022F000BF7FA502000FA102000FA1020064
:10A1A0000FA102000FA102000FA102000FA10200E7
:10A1B0000FA102000FA102000FA102000FA10200D7
:10A1C0000FA102000FA102000FA102000FA10200C7
:10A1D0000FA102000FA102000FA102000FA10200B7
:10A1E0000FA102000FA102000FA102000FA10200A7
:10A1F0000FA102000FA102000FA102000FA1020097
:10A200000FA102000FA102000FA102000FA1020086
:10A210000FA102000FA102000FA102000FA1020076
:10A220000FA102000FA102000FA102000FA1020066
:10A230000FA102000FA102000FA102000FA1020056
:10A240000FA102000FA102000FA102000FA1020046
:10A250000FA102000FA102000FA102000FA1020036
:10A2600063A502000FA102000FA102000FA10200CE
:10A270000FA102000FA102000FA102000FA1020016
:10A280000FA102000FA102000FA1020007A302000C
:10A29000E9A402000FA102000FA102000FA1020019
:10A2A0000FA10200E9A402000FA102000FA1020009
:10A2B0000FA102000FA102000FA102000FA10200D6
:10A2C00051A402000FA102000FA10200C9A30200C5
:10A2D0000FA10200ADA302000FA102000FA1020016
:10A2E00063A5020047F004071C46234613F8012B20
:10A2F0002D2A7FF41DAF47F001071C46F5E747F014
:10A3000002071C46F1E7D9F800301A1DC9F80020F1
:10A310001E78AB680A2E0CD12A68591CA96002F875
:10A3200003B0D5E90123934203D32846FFF710FE7B
:10A33000AB682A68591CA960D654D5E901329A4203
:10A34000FFF4E5AE2846FFF703FE2678002E7FF4E3
:10A35000E2AE2B7B23BB07B0BDE8F08FD9F800201D
:10A36000111DC9F80010166862782E2A04F1020047
:10A370007FF4FEAE5A78A2F13003092B00F2BD81C2
:10A380004FF0000808EB880802EB480810F8012F8E
:10A39000A2F13003092BA8F13008F3D90346E9E60E
:10A3A000284607B0BDE8F04FFFF7D2BDD9F800301E
:10A3B0001A1DC9F8002019680197434600960A2221
:10A3C0002846FFF7E1FDA2E6D9F800301A1DC9F8CA
:10A3D0000020D3F80080FB0700F1E880B8F1000FFF
:10A3E00000F0A181404606F009FF0746BE4215D99C
:10A3F000A6B1202100E08EB1AA682B68501CA8608D
:10A400009954D5E901329A4206F1FF3604D3284621
:10A410000391FFF79DFD0399BE42ECD108F1FF388F
:10A4200018F8016F002E3FF472AEAB6828680A2E50
:10A4300003F1010200EB030100F09081AA600E70AD
:10A44000D5E901329A42EBD32846FFF781FDE7E7D1
:10A45000D9F80020131DC9F80030AB6829681768C7
:10A46000581C3022A860CA54D5E90123934280F0D9
:10A47000E6802A68581C7821A860D154D5E90123C8
:10A48000934280F0D7800F2F03D93A4612090F2A42
:10A49000FCD84FF080560DE0AA6081F80080D5E925
:10A4A00001329A4202D32846FFF752FD36093FF4A3
:10A4B0002EAEAB68B7FBF6F21AF802802868B8F146
:10A4C0000A0F06FB127700EB030103F10102E3D14F
:10A4D000AA6000F803B0D5E901329A4280F04981C0
:10A4E0002B6899180132D7E7D9F800301A1DC9F83E
:10A4F0000020196881EAE173A3EBE173092B40F3B3
:10A500000E81AA480122A0FB03C3DB08092B02F13C
:10A510000102F8DC4245134638BF4346039307F077
:10A520000203002E40F09580002B00F0B780B8F1B8
:10A53000000F00F0F680F80740F1B0800029C0F26B
:10A54000FF807A0700F1C88007F00303022B00F0B8
:10A55000A780CDE9006743460A222846FFF714FD8D
:10A56000D5E5D9F800301A1DC9F8002019680197FF
:10A570004346009610222846FFF706FDC7E5AB6864
:10A580002A68581C2521A860D154D5E901329A4285
:10A59000FFF4BDADD6E6AA6000F803B0D5E90132FC
:10A5A0009A423FD2296811440132A9E54146A1EB04
:10A5B000080311F8017BD7B1AB68D5F800C00A2FAA
:10A5C00003F101020CEB030000F0AF80AA600770FA
:10A5D000D5E901329A42EAD328460391FFF7B8FC45
:10A5E0000399A1EB080311F8017B002FE4D19E42EF
:10A5F0007FF68DAD202702E0002E3FF488ADA968DC
:10A600002A68481CA8605754D5E90121914206F1F7
:10A61000FF3604D328460393FFF79AFC039BB3420B
:10A62000EAD174E52846FFF793FCAB6829685A1C09
:10A63000194465E52846FFF78BFCAB6823E72846FD
:10A64000FFF786FCAB6814E77047184600262346E0
:10A650008BE5002920DB7A071ED41BB1B8F1000F6F
:10A660003FF46CAFF8073FF569AFBEB1039BB3424F
:10A67000BFF464AF2023AA68501CA86028688354E4
:10A68000D5E90102824206F1FF3640D236B1039A83
:10A69000B242F0D1164651E7013EDEE700264DE713
:10A6A000B8F1000F7FF455AF002E6AD0039BB34280
:10A6B000BFF44FAF3023AA68501CA86028688354A9
:10A6C000D5E90102824206F1FF3618D2002E58D099
:10A6D000039AB242EFD13CE7AA68531CAB602B68E7
:10A6E0002B209854D5E901329A42FFF42DAF284629
:10A6F0000491FFF72DFC049926E7034638E5284628
:10A70000CDE90413FFF724FCDDE90413DEE7284656
:10A71000CDE90413FFF71CFCDDE90413B6E70122C1
:10A72000F8E646460AE7474660E6AA600CF803B03A
:10A73000D5E901329A4226D22B689818013245E7B2
:10A74000AA68531CAB602B682D209854D5E90132C0
:10A750009A42C1F10001FFF4F7AEC8E7AA6000F821
:10A7600003B0D5E901329A4217D229681144013267
:10A7700064E62846FFF7ECFBA9682B684A1C1944DD
:10A780008AE60026E5E628460391FFF7E1FBA86884
:10A790002B680399421C184418E72846FFF7D8FB9A
:10A7A000AB6829685A1C194448E600BFCDCCCCCC14
:10A7B000301403002DE9F04182B0002854D0002A63
:10A7C00064D0D0F800C0BCF1000F69D01C46002B4B
:10A7D00033D04768D7F80480B3FBF8F708FB173786
:10A7E000002F3CD18F0723D112F0030F53D1C7683C
:10A7F000B94211D23248334C334B344A3449001BEE
:10A80000C0081024000440F001000094FDF7F6F9A0
:10A81000204602B0BDE8F0814E1E05693444AC42CA
:10A82000E8D8DCF80C40A44602B0BDE8F04160472F
:10A830002348244C244B274AE0E72148214C224B53
:10A84000254A2349001BC0080924000440F00100E8
:10A850000094FDF7D3F9204602B0BDE8F081184816
:10A86000184C194B1D4AECE71548164C164B1C4A60
:10A870001749001BC0080E24000440F0010000949A
:10A88000FDF7BCF9204602B0BDE8F0810C480D4C44
:10A890000D4B144AECE70A480A4C0B4B124AADE741
:10A8A000084C0748084B114A0949001BC0080824F6
:10A8B000000440F001000094FDF7A0F92046A8E74D
:10A8C000842403002424030040140300E41503003F
:10A8D000E8140300A8150300241503007C150300E9
:10A8E000E014030074150300C0150300681503008D
:10A8F000F0B583B0002843D0D0F800C0BCF1000F01
:10A900004ED03AB34768D7F800E00EF1FF370F4258
:10A9100031D1C768B94210D229482A4C2A4B2B4A58
:10A920002B49001BC0081024000440F001000094D3
:10A93000FDF764F9204603B0F0BD4D1E04690EFB1F
:10A940000255A542E8D8DCF81040A44603B0BDE8A3
:10A95000F04060471B4C1A481B4B1E4A1C49001B09
:10A96000C0080924000440F001000094FDF746F9F6
:10A97000204603B0F0BD1248124C134B164ACFE7E5
:10A98000104C0F48104B154A1149001BC0080E24EB
:10A99000000440F001000094FDF730F92046CAE7BA
:10A9A000084C0748084B0E4A0949001BC0080824F8
:10A9B000000440F001000094FDF720F92046BAE7BA
:10A9C000842403002424030054140300901403007F
:10A9D000E81403002415030068140300E0140300C6
:10A9E0006815030029DF704728DF7047034B187A8A
:10A9F0000122B0FA80F05A74400970474C300020B0
:10AA000030B55E4C237A87B0002B3AD05C4B1B6884
:10AA1000022222721A79002A3ED0012A0CD1D3E9EF
:10AA200003021044FFF7E0FF002849D0112803D1AA
:10AA30000123237207B030BD19688A68C2B10022B1
:10AA400068460092C0E902220325026101959A68D6
:10AA500005921A79002A4BD0012A07D102228DF8DB
:10AA60000020DA68120302925B6904938B689847AE
:10AA700000234449444823726360FFF7BFF907B0DD
:10AA800030BD40494048FFF78BF93D4A034610600E
:10AA90000028BDD16060F2E7D3E90525521BB2F56D
:10AAA000805F28BF4FF48052D3E903109208012A37
:10AAB00038BF012229442844FFF794FF0028B5D16C
:10AAC000227C002ADBD1227A002AD8D0022A0AD19D
:10AAD000E0601A79DAB1012A05D1D3E90421013203
:10AAE0008A421A611FD0637C73B102F02FF8C6E767
:10AAF00001228DF800201A690292DA6803925B69DC
:10AB000004938B689847B3E7FFF77AFFB7E7D3E979
:10AB10000512881AB0F5805F94BF121802F58052B2
:10AB200091429A61DFD10022227219688868A8B127
:10AB300068460092C0E90122C0E903229A680592A2
:10AB40001A7982B1012A07D102228DF80020DA6831
:10AB5000120302925B6904938B68984709490A487B
:10AB6000FFF74CF9BFE701228DF800201A69029225
:10AB7000DA6803925B690493EEE700BF4C30002073
:10AB800064300020603000203C30002000F0FD03E5
:10AB9000012B00D0704730B5604CA0F10100B0FA35
:10ABA00080F0237A4009002287B020746274002B61
:10ABB0003AD05B4B1B68022222721A79002A3ED0DF
:10ABC000012A0CD1D3E903021044FFF70DFF00283E
:10ABD00049D0112803D10123237207B030BD196871
:10ABE0008A68C2B1002268460092C0E902220325A9
:10ABF000026101959A6805921A79002A4BD0012AC0
:10AC000007D102228DF80020DA68120302925B69F4
:10AC100004938B689847002342494348237263603A
:10AC2000FFF7ECF807B030BD3E493F48FFF7B8F8F2
:10AC30003B4A034610600028BDD16060F2E7D3E9CB
:10AC40000525521BB2F5805F28BF4FF48052D3E92F
:10AC500003109208012A38BF012229442844FFF733
:10AC6000C1FE0028B5D1227C002ADBD1227A002A3D
:10AC7000D8D0022A0AD1E0601A79CAB1012A05D1D6
:10AC8000D3E9042101328A421A611DD0637C63B189
:10AC900001F05CFFC6E701228DF800201A690292DC
:10ACA000DA6803925B690493B3E7FFF7A9FEB9E79B
:10ACB000D3E90512881AB0F5805F94BF121802F527
:10ACC000805291429A61E1D100222272196888680B
:10ACD000A8B168460092C0E90122C0E903229A683F
:10ACE00005921A7982B1012A07D102228DF800203B
:10ACF000DA68120302925B6904938B6898470949EA
:10AD00000948FFF77BF8C1E701228DF800201A6996
:10AD10000292DA6803925B690493EEE74C300020FC
:10AD200064300020603000203C300020831E012B66
:10AD300000D9704730B58E4C237A87B0002B31D0C4
:10AD4000022B2BD103286BD1E3680133082B79D96F
:10AD5000884B00221B68E26022720D2519688A6800
:10AD6000C2B1002268460092C0E902220261019548
:10AD70009A6805921A79002A00F0B980012A07D151
:10AD800002228DF80020DA68120302925B690493B4
:10AD90008B68984778497948FFF730F8637C1BB196
:10ADA00001F0D4FE07B030BD237A002B5BD0714B8D
:10ADB0001B68022222721A79002A5FD0012A0BD165
:10ADC000D3E903021044FFF70FFE002869D01128D1
:10ADD00002D101232372E5E719688A68C2B1002213
:10ADE00068460092C0E902220325026101959A6833
:10ADF00005921A79002A70D0012A07D102228DF813
:10AE00000020DA68120302925B6904938B6898470A
:10AE100000235949594823726360FEF7EFFFC1E7E9
:10AE2000544B00221B68E2601A796AB1012AB5D13D
:10AE3000D3E9042101328A421A6111D0637C002BCC
:10AE4000AED1B4E7E360F9E7D3E90512881AB0F5AB
:10AE5000805F94BF121802F5805291429A61EDD141
:10AE6000002525727AE744494448FEF799FF414A94
:10AE70000346106000289CD1606093E7D3E9052564
:10AE8000521BB2F5805FD3E9031028BF4FF4805204
:10AE90009208012A38BF012229442844FFF7A2FD65
:10AEA00093E7227C002A7FF47DAF227A002A3FF4C8
:10AEB00079AF022A0AD1E0601A7912B3012A05D1CA
:10AEC000D3E9042101328A421A6126D0637C002B27
:10AED0007FF466AFFFF794FD64E701228DF8002050
:10AEE0001A690292DA6803925B6904938EE7012281
:10AEF0008DF800201A690292DA6803925B69049364
:10AF000046E7D3E90512881AB0F5805F94BF12189E
:10AF100002F5805291429A61D8D1002222721968BA
:10AF20008868A8B168460092C0E90122C0E90322FE
:10AF30009A6805921A7982B1012A07D102228DF806
:10AF40000020DA68120302925B6904938B689847C9
:10AF500009490A48FEF752FFB8E701228DF80020A0
:10AF60001A690292DA6803925B690493EEE700BF04
:10AF70004C30002064300020603000203C30002045
:10AF8000FEF786BF2DE9F041058ACE1C043D2E4414
:10AF90000746B6FBF5F6FEF797FF78B3F6B24FF427
:10AFA0008073013E0446C5800760838027D08046B9
:10AFB000002509E06379AE4203F101036371C8F82B
:10AFC0000000076080461AD03846FEF77DFF013545
:10AFD0000028EFD16679721E14D0234601308242D8
:10AFE0001B68FBD11F684EB100252368214601353F
:10AFF00038461C46FEF790FFAE42F6D100242046AC
:10B00000BDE8F0812768EFE704300121FEF710BFAB
:10B01000F8B5012104460430FEF716FFC0B200B1B6
:10B02000F8BD6679721E12D02346013082421B6839
:10B03000FBD11F68002EF3D000252368214601357F
:10B0400038461C46FEF768FFAE42F6D1F8BD2768C9
:10B05000F2E700BF2DE9F843C788467907FB06F6FB
:10B06000043E02EB030C0446664503F1040015465A
:10B070008846B0FBF7F238BFF51A07FB120012B191
:10B08000013A2468FCD13E1AAE4228BF2E469DB13B
:10B090004FF000090430AD1B2044324608EB090193
:10B0A00006F099F8AF42B14424683E464FF00000E4
:10B0B00028BF2E46002DEDD1BDE8F8832DE9F843D9
:10B0C000C7884679154607FB06F6043E05EB030CD8
:10B0D0001A1D664504468846B2FBF7F038BFF51ADC
:10B0E00007FB102110B101382468FCD17E1AAE4252
:10B0F00028BF2E469DB14FF0000904312144AD1BFD
:10B10000324608EB090006F066F8AF42B144246805
:10B110003E464FF0000128BF2E46002DEDD1BDE880
:10B12000F88300BF8268002393608268136182689D
:10B1300053618268D360826853608268136070478D
:10B1400001600B6843604A68934204BF0023436078
:10B15000704700BF436843B1026891680B44436085
:10B160005268934204BF00234360704770B544683F
:10B17000064620680D4618B908E02468206828B102
:10B18000B368294698470028F7D1206828602560D1
:10B1900070BD00BF4368186808B102681A60704744
:10B1A00043681868704700BF4068036873B18B42FA
:10B1B00003D107E0814204D0034618680028F9D182
:10B1C000704718460B6803600120704718467047A7
:10B1D00030B4184DA5F59472AB1ADB1003EBD373A2
:10B1E0005B1002EBC30152F83330984228BF0C4683
:10B1F00005D311E052F8333098420CD221468B1A15
:10B20000DB1003EBD3735B108A4202EBC304F1D370
:10B21000094830BC70470D46984204D904F1080231
:10B22000AA42D9D3F4E76068034B002808BF184648
:10B23000EFE700BF641703002816030010B570B1D4
:10B2400001280BD10D4C2369A0703BB1D3E9002339
:10B250000120226198472369002BF7D110BD074CCC
:10B26000A36801226270002BF8D0D3E900230020EC
:10B27000A2609847A368002BF7D1EFE76830002061
:10B2800070B910B5074CA368012262703BB1D3E9D5
:10B2900000230020A2609847A368002BF7D110BDBF
:10B2A000704700BF6830002030B5012883B01CD043
:10B2B00015D3032811D100F0CDF802A800231F4CAC
:10B2C00000F8013DFDF7CEFDE368013BE360E56872
:10B2D00065B39DF80700FDF7EBFD03B030BD184BDB
:10B2E0000122C3F8802003B030BD02A80023134C14
:10B2F00000F8013DFDF7B6FD237853B1E3689DF8F2
:10B30000070001330122E360A270FDF7D1FD03B015
:10B3100030BD0C486360A3602361E36000F08CF8EB
:10B3200001F024FC30B101232370E7E700F0A4F81A
:10B33000A570CEE700F08EF8F5E700BF683000207A
:10B3400000E100E03DB2020030B585B00478456808
:10B350008DF80040D0E90240064A074B039053F8AD
:10B36000213001958DF8084052F821106846984721
:10B3700005B030BD7C3000208430002030B585B071
:10B38000047845688DF80040D0E90240064A074B32
:10B39000039053F8213001958DF8084052F82110A0
:10B3A0006846984705B030BD7C30002084300020CE
:10B3B0002DE9F043DFF8748006784B7F08F80630FB
:10B3C0000D46074696460FCD89B06C460FC495E8EA
:10B3D0000F003D78DFF85890DFF858C018F8055096
:10B3E00049F826E084E80F004CF82600049665B181
:10B3F000BEF1000F0B4A694607F1040008BF0022A6
:10B4000001F094F809B0BDE8F083BEF1000F064AE0
:10B41000694607F10C0008BF002200F007FE09B0E2
:10B42000BDE8F08349B302007DB30200305800202C
:10B43000843000207C300020054A13792BB901218B
:10B44000106053711846117170478520704700BF16
:10B450008C300020074B1A68D20704D4C021012287
:10B4600083F800131A604FF080430122C3F81825B7
:10B47000704700BF00E100E0044B01221A604FF06A
:10B480008042D2F81834DB03FBD470470C00004034
:10B4900010B5154B1A6882B07AB10021134A1960B1
:10B4A0001B68507900934FF080410123009CC1F844
:10B4B000083310B91168537188470D4B1A6882B16F
:10B4C00000221A601B6801934FF080420221074B53
:10B4D0000198C2F808131B68012002B0BDE81040B3
:10B4E000184702B010BD00BF000100408C300020A2
:10B4F0000401004030B5204C94F86A5083B0002D10
:10B5000036D14FF0FF332946062204F16400C4E926
:10B510000033C4E90233C4E90433C4E90633C4E99F
:10B520000833C4E90A33C4E90C33C4E90E33C4E96F
:10B530001033C4E91233C4E91433C4E91633236663
:10B5400005F054FE0D4A0E4B0E491D60C02082F8D6
:10B550000603402010601B68019301984FF00043E0
:10B560000122284684F86A20C1F8043303B030BDB4
:10B57000082003B030BD00BF9430002000E100E09F
:10B580007C61004000600040034B93F86A0000308B
:10B5900018BF0120704700BF94300020F0B5744BF5
:10B5A0001C1894F93050002D6ADA8E78C6F34006E4
:10B5B0009646002E5ED11D6A013500F0C480092434
:10B5C0000C2553F8247001375DD004F1010C53F8B9
:10B5D0002C70013700F0C280A71CAF4248D253F84C
:10B5E0002720013200F0BC8004F1030CAC453FD2AF
:10B5F00053F82C70013700F0B18004F1040CAC4515
:10B6000036D253F82C70013700F0A88004F1050CF5
:10B61000AC452DD253F82C70013700F09F8004F117
:10B62000060CAC4524D253F82C70013700F09680FC
:10B6300004F1070CAC451BD253F82C70013700F015
:10B640008D8004F1080CAC4512D253F82C700137F0
:10B6500000F0848004F1090CAC4509D253F82C7039
:10B6600001377BD00A34AC4202D2DC6A013409D003
:10B670000420F0BD1D68013574D001240825A0E721
:10B680000820F0BD0B241F1865B243F824E087F8AA
:10B690003050002E5ED08A7854071AD4D60741D491
:10B6A0001F284A7887BF334E00F01F0404464FF02E
:10B6B000A04604F5E074920046F824202E4EC408FB
:10B6C00000F0070C375D012202FA0CF23A433255C2
:10B6D0008A780C7812F0020209D1083D2B441046FA
:10B6E00093F8602042EA841483F86040F0BDAB0018
:10B6F00003F1804303F5C0430202D3F8101521F48F
:10B700004F3121F44071C3F810152404D3F81015FB
:10B7100004F4403402F47C5222430A43C3F8102557
:10B720000020F0BD1F2887BF124A00F01F04044606
:10B730004FF0A04202EB8402D2F8004724F002044A
:10B74000C2F80047BAE7082684F83060C3F820E062
:10B75000354634461C4484F858009CE7644692E71A
:10B760003C4690E700251A6084F8305093E700BF0C
:10B770009430002000030050F830002070B43A4D9F
:10B780002E1883B096F93030072B20DD2B4493F828
:10B7900058309B09032B45D0012B14BF4FF4403187
:10B7A0004FF400311F284DD900F01F002F4B03EB41
:10B7B0008000D0F8002722F44032C0F80027D0F8EB
:10B7C00000370B43C0F8003703B070BC7047DAB2E3
:10B7D000072AF9D8980000F1804000F5C04003F135
:10B7E0004002D0F81045920092B244F0010402F1F8
:10B7F0008042C0F8104502F5C04200200190019C33
:10B8000010600029E0D096F9302055F82220002A57
:10B81000DAD00122164902FA03F3C1F8043303B067
:10B8200070BC70471F2810D9104BD3F8103500F0AA
:10B830001F00C34013F0010F0CBF4FF400314FF451
:10B840004031B3E74FF0A043B1E74FF0A0421346B9
:10B85000D2F81025C24012F0010F14BF4FF440314E
:10B860004FF40031A3E700BF9430002000030050E4
:10B87000006000401F288ABF054B4FF0A04300F036
:10B880001F00D3F8103523FA00F000F001007047D4
:10B89000000300502DE9F047002388B0CDE90233C2
:10B8A000CE4A1668012E00F03B821E46CC4B1A6829
:10B8B000012A00F02782CB4B1A68012A00F014827B
:10B8C000C94B1A68012A00F00182C84B1A68012A84
:10B8D00000F0EE81C64B1A68012A00F0DB81C54BEF
:10B8E0001A68012A00F0C881C34B1A68012A00F0C7
:10B8F000B581C24B1A68012A0FD100221A601B6859
:10B9000001934FF0A042019BD2F81025BC4B02924C
:10B91000D3F81035039346F0004616F0FF0F1AD007
:10B92000B84F00240125A30003F180432E4203F504
:10B93000C0434FEA45050BD0D3F8100557F8242033
:10B94000D3F81015C0F30520C1F3014102B19047AF
:10B950000134082CE7D1002E02DB08B0BDE8F087E7
:10B96000A84CA74F4FF0FF33CDE9063394F9603070
:10B970000DF1100800225D1CC8F8042004924FF05D
:10B98000010600F0F4805FFA83FC2CF0C00008ABE5
:10B990004FEAD00903EB090E0CF007031EF8082C40
:10B9A00006FA03F312EA030521D022184FEA9C118C
:10B9B00092F9302054F82220002A00F0298103292E
:10B9C00000F028811F2800F2F98005464FF0A04CB6
:10B9D0000CEB850C1EF8185CDCF800E71D40CEF37C
:10B9E000014E40F0DF80BEF1030F00F0BF8194F9FB
:10B9F0006130581C32D0DBB223F0C00008AA4FEAF5
:10BA0000D00E02EB0E0C03F007011CF8082C06FA0E
:10BA100001F912EA090F21D02218990992F9302070
:10BA200054F82220002A00F0FB80032900F0FB805C
:10BA30001F2800F2E98003464FF0A04E0EEB83036F
:10BA40001CF818ECD3F800C71EEA090FCCF3014C20
:10BA500040F0B880BCF1030F00F0AE8194F9623081
:10BA6000591C30D0DBB223F0C00008AA4FEAD00E38
:10BA700002EB0E0C03F007011CF8082C06FA01F982
:10BA800012EA090F1FD02218990992F9302054F8B0
:10BA90002220002A00F0D880032900F0D8801F2837
:10BAA0007CD803464FF0A04E0EEB83031CF818EC35
:10BAB000D3F800C71EEA090FCCF3014C64D1BCF1E6
:10BAC000030F00F0658194F963305A1C34D0DBB267
:10BAD00023F0C00008AA4FEAD00E02EB0E0C03F0D0
:10BAE00007021CF8081C06FA02F2114224D004EBEB
:10BAF0000009990999F9309054F82990B9F1000F8B
:10BB000000F09880032900F098801F288BBFBE4664
:10BB10004FF0A04E03F01F0303460EEB83031CF807
:10BB200018ECD3F800C71EEA020FCCF3014C20D169
:10BB3000BCF1030F00F00181002D3FF40EAF4FF078
:10BB4000A0430299D3F81035D7F81025994203D1B4
:10BB5000039991423FF401AFDDE90401CDE90232DE
:10BB600094F960305D1CCDE906017FF40CAF00252F
:10BB70003DE7BCF1020FDFD1032900F03481B9F1B8
:10BB8000000F40F0F180D7E7BCF1020F9BD10329F1
:10BB900000F02681002A96D0904794E703F01F0317
:10BBA000BE4681E7BEF1020FE1D1032900F02181F9
:10BBB0000025002A3FF41BAF904718E70CF01F0543
:10BBC000BC4605E7BCF1020F7FF448AF032900F043
:10BBD0000D81002A3FF442AF90473FE700610040EB
:10BBE00004610040086100400C61004010610040A9
:10BBF00014610040186100401C6100407C610040FD
:10BC0000000300509430002003F01F03BE4615E7E8
:10BC10000329ACD118F809501D4308F80950D1E6A2
:10BC200003297FF41BAF18F80EA04AEA090A08F8A6
:10BC30000EA0FDE603297FF47FAF18F80EA04AEAB4
:10BC4000020A08F80EA060E703297FF43CAF18F859
:10BC50000EA04AEA090A08F80EA020E7664AD2F8C0
:10BC6000042317067FF545AE00221A601B68009377
:10BC7000009B46F080063CE65F4AD2F80423520659
:10BC80007FF532AE00221A601B680093009B46F0DD
:10BC9000400629E6584AD2F8042391067FF51FAEE4
:10BCA00000221A601B680093009B46F0200616E6EF
:10BCB000514AD2F80423D0067FF50CAE00221A6058
:10BCC0001B680093009B46F0100603E64A4AD2F830
:10BCD000042314077FF5F9AD00221A601B68009356
:10BCE000009B46F00806F0E5434AD2F804235507C6
:10BCF0007FF5E6AD00221A601B680093009B46F0BA
:10BD00000406DDE53C4AD2F8042397077FF5D3AD5E
:10BD100000221A601B680093009B46F00206CAE5E9
:10BD20003549D1F8041311F0010104D013601368F0
:10BD30000093009BBAE50E46B8E503297FF41FAFD8
:10BD40004FF4003CD3F8002722F44032C3F8002718
:10BD5000D3F80027013542EA0C02EDB2C3F8002700
:10BD6000B9F1000F3FF4EBAEC847E5E603297FF4D5
:10BD700020AF4FF40035DCF8003723F44033CCF823
:10BD80000037DCF800372B43CCF80037012510E7EB
:10BD900003297FF4FFAE4FF4003ED3F800C72CF424
:10BDA000403CC3F800C7D3F800C701354EEA0C0C7D
:10BDB000EDB2C3F800C7EDE603297FF40AAF4FF4F4
:10BDC000003ED3F800C72CF4403CC3F800C7D3F8BA
:10BDD00000C701354EEA0C0CEDB2C3F800C7F8E617
:10BDE0004FF4403ED9E74FF4403CABE74FF4403EC0
:10BDF000E7E74FF44035BEE700600040014B1B68A9
:10BE0000184700BF00310020104B984201D000209D
:10BE1000704730B583B002A8002300F8013D0D46FD
:10BE2000FDF720F80A4B1C7934B19DF80700FDF7A7
:10BE30003FF8112003B030BD01229DF807001D60BE
:10BE40001A71FDF735F82046F4E700BF00200040E6
:10BE500000310020034B984203D1034B00221A60AB
:10BE60001A717047002000400031002030B56D4A43
:10BE7000D2F8043399058BB068D5D2F82431002B61
:10BE800064D00023C2F82431D2F8243101934FF456
:10BE90000171654B0198C2F8081393F8291009B98C
:10BEA000012151605F4902228DF81820D1F88024C9
:10BEB000C1F880249869D96809920022CDE9071059
:10BEC000C3E90622D3E9001406A8A047554AD2F8D0
:10BED0001C31CBB1544B5869196A88426BD851490F
:10BEE0000022C1F81C21D1F81C1102910299596954
:10BEF00051B1586999688DF8182008905A610791D6
:10BF000006A8D3E900129047464AD2F84431DBB183
:10BF10000021454BC2F84411D2F8440193F829108E
:10BF20000090009809B1012111609A6962B1002264
:10BF3000586AD9689A610122CDE907108DF8182056
:10BF400006A8D3E9001290470BB030BD354AD2F8AD
:10BF500004335B07BAD5D2F80831002BB6D0324B88
:10BF6000996900293CD00021C2F80811D2F80811C3
:10BF700004910499D868596AD2F8182542545A6A2B
:10BF8000996901325A625A6A8A429FD1DA691968FC
:10BF9000002A2ED0D8685D6A1C699A610790002239
:10BFA0000120DC60DA615A628DF8180008955B6840
:10BFB00006A898478AE793F8281001F0FF000029A7
:10BFC0008DD1C2F81C01D2F81C11039103999C6811
:10BFD000186A196A205C01311962C2F81C0593E7DE
:10BFE000C2F80811D2F8080105900598D2F8182572
:10BFF000C9E793F8292012B90A4A01205060094A7A
:10C000004FF40170C2F80803586ADA6808900024F7
:10C01000012007928DF818005A689C6106A8904785
:10C0200054E700BF00200040083100202DE9F04116
:10C03000714F06792C2505FB067582B095F82A30DC
:10C04000002B40F09A800D4604466C4900689046EB
:10C05000FFF7DAFE002840F08C802B68591C19D0BD
:10C060001F2B4FF001028ABF65494FF0A04103F03A
:10C070001F0302FA03F3C1F808352B681F2B86BF94
:10C0800003F01F035E4A4FF0A04203F5E073032163
:10C0900042F823106B685A1C0BD01F2B86BF03F08D
:10C0A0001F03574A4FF0A04203F5E073002142F806
:10C0B00023102368AA69C3F82425297D6B7D226893
:10C0C0000B43C2F86C35D5E900122368C3F8142578
:10C0D000C3F80C152B7D012B53D02C2303FB06F347
:10C0E000FA18C2F804802A69FA50B8F1000F2DD06E
:10C0F00022682B7F434D0021C2F81C11D2F81C216D
:10C1000000922268DDF800C0C2F84411D2F8441150
:10C11000226801910199C2F804532168090B4AB2BF
:10C120005B01002ADBB261DB02F1604202F5614291
:10C1300082F800332368344D1B0B5AB2520903F0C6
:10C140001F03012101FA03F345F822302C23246850
:10C1500003FB0673002204250121C4F8005583F86F
:10C160002A10C3E9062283F829205A6102B0BDE8EB
:10C17000F081112002B0BDE8F081082002B0BDE8D6
:10C18000F081AB68591C0BD01F2B86BF03F01F0337
:10C190001B4A4FF0A04203F5E073002142F8231040
:10C1A000EB685A1C1BD01F2B4FF001028ABF1449A9
:10C1B0004FF0A04103F01F0302FA03F3C1F8083562
:10C1C000EB681F2B88BF03F01F0303F5E0738CBFE0
:10C1D0000B4A4FF0A042032142F82310EB6822687B
:10C1E000A968C2F80835C2F8101576E7074A01F0C9
:10C1F0000F010A4413769DE7083100206DBE02004E
:10C20000000300508000020000E100E0FCEC00E0D0
:10C21000F8B53A4F047902682C2303FB047300211C
:10C220005B68C2F8001583B10368354AC3F8082378
:10C230000368344D1B0B5AB25209203203F01F031E
:10C24000012101FA03F345F8223003684FF0FF3C67
:10C25000D3F80C65D3F81455D3F80825D3F8101586
:10C26000C3F814C5C3F80CC503686645C3F808C510
:10C27000C3F810C50CD01F2E86BF06F01F06224B38
:10C280004FF0A04306F5E0764FF0020C43F826C0CD
:10C290006E1C0BD01F2D86BF05F01F051A4B4FF0EB
:10C2A000A04305F5E075022643F825604D1C0BD030
:10C2B0001F2986BF01F01F01134B4FF0A04301F56A
:10C2C000E071022543F82150531C0BD01F2A86BF72
:10C2D00002F01F020C494FF0A04102F5E072022368
:10C2E00041F822300068FFF7B5FD2C2303FB0474EE
:10C2F000002384F82A306360F8BD00BF08310020B5
:10C300008402020000E100E000030050F0B5314E6D
:10C3100005792C2303FB056385B05C69002C53D1A0
:10C320005A6199601C6283F828400268C2F81C4177
:10C33000D2F81C11026802910121029F91600268EB
:10C34000D3F808C0C2F81C41D2F81C110191019920
:10C35000D3F820E0196A5F681CF80EE00131196219
:10C36000C2F81CE517B1204605B0F0BD5C691A6A39
:10C370000168944203D819E093F828203ABBD1F819
:10C380001C21002AF8D0C1F81C71D1F81C2103929D
:10C39000039AD3F820E01A6A1CF80EE001321A6200
:10C3A000C1F81CE51A6A9442E9D80168D1F81C3139
:10C3B000002BFBD00123CB6000202C2303FB056561
:10C3C00000236B6105B0F0BD112005B0F0BD0F205A
:10C3D000F3E700BF08310020F0B5524BD3F8242119
:10C3E0008BB0002A6ED00021C3F82411D3F8242189
:10C3F000049202228DF81820049AD3F880044A4A45
:10C40000C3F880040990D3F83C05D3680890C2E9CA
:10C41000061107931168536806A89847414BD3F853
:10C420004421BAB10021404AC3F84411D3F8444131
:10C4300090690394039C68B1D3F83C35D0680893A5
:10C440000123C2E9061107908DF8183006A8D2E939
:10C4500000139847334BD3F82021BAB10021C3F819
:10C460002011D3F82021029201202F4A029CD8608B
:10C47000506958B1D3F84C05936808908DF818109E
:10C480005161079306A8D2E900139847254BD3F8CA
:10C490005821AAB10021C3F85811D3F85801224AF3
:10C4A00001900198506958B1D3F84C0593680890F1
:10C4B0008DF818105161079306A8D2E90013984728
:10C4C0000BB0F0BDD3F810110029A7D0C3F810218C
:10C4D000D3F810111448059105998169D3F83C45AA
:10C4E0008C429BD1C569C768D0E900168DB1D3F8DD
:10C4F00000C285612CF02005C261C3F800520369B7
:10C50000C3600122CDE907748DF8182006A8B04752
:10C5100084E701238561CDE907748DF8183006A8FA
:10C52000B0477BE700200040343100202DE9F04384
:10C5300007797E4E4FEAC70808EB070306EB830333
:10C5400087B093F82030002B40F0B0800D460446B1
:10C55000774900689146FFF757FC002840F0A28019
:10C560002B68591C19D01F2B4FF001028ABF71494B
:10C570004FF0A04103F01F0302FA03F3C1F808359E
:10C580002B681F2B86BF03F01F036A4A4FF0A0429F
:10C5900003F5E073032142F823106B685A1C0BD09B
:10C5A0001F2B86BF03F01F03624A4FF0A04203F522
:10C5B000E073002142F823102368AA69C3F82425F8
:10C5C000297D6A7D23680A43C3F86C25D5E90031CB
:10C5D0002268C2F80C35C2F814152B7D012B69D0E6
:10C5E00008EB07029200B318C3F804902B69B3500C
:10C5F000B9F1000F45D021682A7F4F4D0023C1F8C3
:10C600001031D1F8101101912168DDF804C0C1F892
:10C610002031D1F8201102912168DDF808C0C1F85D
:10C620002431D1F8241103912168DDF80CC0C1F840
:10C630004431D1F8441104912168DDF810C0C1F8EB
:10C640005831D1F85811236805910599C3F804535E
:10C650002168090B53014AB2002ADBB25FDB02F109
:10C66000604202F5614282F800332368334D1B0BB0
:10C670005AB2520903F01F03012101FA03F345F8EE
:10C6800022304744226806EB870600230124082154
:10C69000C2F8001586F82040C6E90633736107B07A
:10C6A000BDE8F083112007B0BDE8F083082007B093
:10C6B000BDE8F083AB68591C0BD01F2B86BF03F07D
:10C6C0001F031C4A4FF0A04203F5E073002142F81B
:10C6D0002310EB685A1C1BD01F2B4FF001028ABF9E
:10C6E00014494FF0A04103F01F0302FA03F3C1F80D
:10C6F0000835EB681F2B88BF03F01F0303F5E073B9
:10C700008CBF0C4A4FF0A042032142F82310EB6883
:10C710002268A968C2F80835C2F8101560E7084A0F
:10C7200001F00F010A4413769FE700BF3431002067
:10C73000D9C30200000300501003420000E100E0F2
:10C74000FCEC00E0F0B50679474C0368F500AA1947
:10C7500004EB820283B0526882B1444AC3F80823D2
:10C760000368434F1B0B5AB25209203203F01F03D8
:10C77000012101FA03F347F822300368D3F80022BD
:10C7800022F02002C3F800220268012353600268ED
:10C790000021C2F85811D2F858110268019101998C
:10C7A000D3600268D2F85831002BFBD00023C2F8C6
:10C7B000003503684FF0FF3ED3F80CC5D3F814756D
:10C7C000D3F80825D3F81015C3F80CE5C3F814E521
:10C7D0000368F445C3F808E5C3F810E50DD0BCF1D3
:10C7E0001F0F86BF0CF01F0CDFF888E04FF0A04E43
:10C7F0000CF5E07C02234EF82C307B1C0CD01F2F54
:10C8000086BF07F01F07DFF86CC04FF0A04C07F59C
:10C81000E07702234CF827304F1C0BD01F2986BF2E
:10C8200001F01F01134F4FF0A04701F5E071022303
:10C8300047F82130531C0BD01F2A86BF02F01F027D
:10C840000C4B4FF0A04302F5E072022143F8221096
:10C850000068FFF7FFFA354404EB8504002384F8F1
:10C860002030636003B0F0BD34310020100342007B
:10C8700000E100E00003005001F06043B3F1005F0D
:10C880002CD1F0B40579264EEF007C1906EB840418
:10C8900082B0636923BB6261A1600268C2F8203183
:10C8A000D2F820C10268CDF804C0DDF804C0C2F897
:10C8B0005831D2F8582100920268DDF800C0D4F84F
:10C8C00014C0C2F84415C2F848C50268012191603D
:10C8D00062684AB1184602B0F0BC70471020704739
:10C8E000112002B0F0BC7047036800E0B2B9D3F881
:10C8F0002011D3F858210029F8D07AB90122DA6042
:10C900000268D2F85831002BFBD000203D4406EBE2
:10C9100085060023736102B0F0BC70470F20F5E775
:10C920003431002010DF704711DF704700B583B04D
:10C9300068460849FEF704FC019B43B1D3E9002097
:10C9400090476846FEF706FC019B002BF6D103B02A
:10C950005DF804FB8C1B030070B53B4D2B7884B055
:10C96000002B63D1394E3A49012302A83370FEF7F8
:10C97000E7FB039B002B4FD1364902A8FEF7E0FBF3
:10C98000039B4BB1D3E900210020904702A8FEF79A
:10C99000E1FB039B002BF5D12F4A002312688DF891
:10C9A000083002A80192FCF75DFA2C4901A8FFF7B4
:10C9B000B9FFB0FA80F304465B099DF808002B70BC
:10C9C000FCF776FA002C2ED1254B26491C703470CA
:10C9D00091F81623EC2352091341DB072FD5224B84
:10C9E0009A683ABB4FF480030B601A4902A8FEF71D
:10C9F000A7FB039BBBB1D3E900210120904702A80C
:10CA0000FEF7A8FB039B002BF5D10CE002A8FEF774
:10CA1000A1FB039B002BAFD0D3E90021002090475E
:10CA20000028F3D10446204604B070BD08242046F7
:10CA300004B070BD1A6842F480021A60D5E742F271
:10CA40000200FBF783FED0E7593100205831002067
:10CA5000801B0300981B03007C1B03006D870200F2
:10CA60005A31002000E100E024580020F0B5314D9B
:10CA70002B7883B0002B54D02F4E304901236846C9
:10CA80003370FEF75DFB019B002B40D12C496846BB
:10CA9000FEF756FB019B4BB1D3E9002102209047E2
:10CAA0006846FEF757FB019B002BF5D1002768462F
:10CAB0008DF80070FCF7D6F9FFF736FF04469DF8B5
:10CAC00000002F70FCF7F4F944BB1E4B34709A68D9
:10CAD0005ABB1D4B4FF48002C3F8802018496846AA
:10CAE000FEF72EFB019BCBB1D3E900210320904739
:10CAF0006846FEF72FFB019B002BF5D1204603B0C3
:10CB0000F0BD6846FEF726FB019B002BBED0D3E9A3
:10CB10000021012090470028F3D10446204603B0AD
:10CB2000F0BD0824204603B0F0BD1A6822F480024C
:10CB30001A60D3E75931002058310020801B0300D0
:10CB4000981B03002458002000E100E0054B1B78EF
:10CB500033B1054B1B780BB9FFF7FEBEFFF786BF5D
:10CB6000082070475831002059310020014B1878B7
:10CB7000704700BF59310020002108B50846044A1B
:10CB8000FBF754FE00B908BDBDE80840FBF7DEBD69
:10CB90002DC9020060DF704761DF7047134B1B78BF
:10CBA0001BB330B5124D91B034240DF1020103A82E
:10CBB000ADF80240FFF7F0FF88B9294601A8FEF75B
:10CBC000BFFA029B002BF0D0D3E9002103A89047C5
:10CBD00001A8FEF7BFFA029B002BF5D1E5E7052877
:10CBE00001D0FBF7B3FD11B030BD70475B310020C1
:10CBF0005C1C030018B1034B0360002070470E203B
:10CC0000704700BF681F0020F8B506460768FFF7A9
:10CC1000C1FF3368BB42054605D825BB1A4B01222C
:10CC20001A702846F8BD194B194C1A49E41AE40841
:10CC3000240444F002042046FAF730FD3A46204628
:10CC400033681549FAF758FF4FF080533268D3F82C
:10CC50000C3112499B0203F1005320469A1AFAF74D
:10CC6000CBFE002DDAD02846FEF7B2FA074A084B71
:10CC70000B499B1ADB081B04024643F00100FAF73C
:10CC8000BBFE2846F8BD00BF5B3100202424030012
:10CC900094240300AC1B0300DC1B0300101C0300E6
:10CCA0003C1C03004BDF704710B5114C84B001A849
:10CCB000FFF7F8FFA8B9214602A8FEF741FA039B47
:10CCC000002BF4D0D3E900210198904702A8FEF789
:10CCD00041FA039B002BF5D101A8FFF7E3FF0028E1
:10CCE000E9D0052801D0FBF731FD04B010BD00BF2D
:10CCF000741C030041DF704730B43D4A1378042BA5
:10CD00001CD8DFE803F0133A1F32030039490878D2
:10CD100004284AD04FF0A0424FF408140020C2F873
:10CD20000845C2F80C050B7030BC70474FF0A042AC
:10CD30003149C2F808150021C2F80C152D490B70B5
:10CD400030BC70474FF0A0424FF4800100204FF4F8
:10CD50000C14C2F80C152749C2F80805C2F808459A
:10CD6000C2F80C050B7030BC70474FF0A0424FF476
:10CD7000803100204FF4C404EBE74FF0A0421D497E
:10CD8000D2F80405C44304F48004C2F808454FF403
:10CD90000C15002400F48000C2F80C05C2F80855F8
:10CDA000C2F80C450B7030BC7047144C2078013031
:10CDB000C0B2042820700CD94FF0A04303204FF4D8
:10CDC00008150024C3F80855C3F80C450346107035
:10CDD000A9E74FF0A040D0F80425D44304F4081488
:10CDE00002F40812C0F80845C0F80C259BE700BF04
:10CDF000AD3E0020E03E00200000E301AC3E0020FC
:10CE0000704700BF70B5184B184CE41AE4082404AE
:10CE100005460E4644F0030420462A461449FAF714
:10CE2000EBFD3378012B12D007D3022B0ED1204615
:10CE30001049BDE87040FAF731BC20460E49FAF7B8
:10CE40002DFC0E4A0E4B156003221A7070BD204651
:10CE50000C490A4CFAF722FC0B48094A002302212C
:10CE600023600370117070BD242403004C24030060
:10CE7000A01F030000200300D41F0300DC3E00209D
:10CE8000AD3E0020EC1F0300D83E00202DE9F0410C
:10CE9000704C714D2D1BED082D0445F0030682B03A
:10CEA00090460C4602461F4630466C49FAF7A4FDF0
:10CEB000002F40F087806A493046FAF7EFFB45F0D3
:10CEC0000505E07AA17A637A227A019000912846DA
:10CED0006449FAF71BFFE07BA17B637B227B019017
:10CEE000009128465F49FAF711FFE07CA17C637C42
:10CEF000227C0190009128465A49FAF707FFE07D0D
:10CF0000A17D637D227D0190009128465649FAF764
:10CF1000FDFE56493046FAF7C1FBE07EA17E637EF6
:10CF2000227E0190009128464E49FAF7EFFEE07FFD
:10CF3000A17F637F227F0190009128464949FAF73B
:10CF4000E5FE94F8230094F8221094F8213094F828
:10CF500020200190009128464249FAF7D7FE94F824
:10CF6000270094F8261094F8253094F82420019096
:10CF7000009128463C49FAF7C9FE3A463C493046FA
:10CF8000FAF73AFD98F80030802B5ED00BD9862B4B
:10CF900052D01BD8812B3AD0852B0FD13046354942
:10CFA000FAF77CFB0AE0022B41D039D9032B29D0B8
:10CFB000042B03D130463049FAF770FB002002B051
:10CFC000BDE8F0813846FBF7C1FB74E7872B14D02E
:10CFD000882BF3D130462949FAF760FB284B1A78A1
:10CFE000002AEBD02749284C04200022087000209A
:10CFF00022701A7002B0BDE8F08130462349FAF77A
:10D000004DFBDBE730462249FAF748FBD6E73046CE
:10D010002049FAF743FB1A4B1A78002ACED0E1E7F1
:10D02000012BCBD130461C49FAF738FBC6E7304616
:10D030001A49FAF733FBC1E730461949FAF72EFBD4
:10D040000F4B1A78002ACDD1B8E730461549FAF7C8
:10D0500025FBB3E7242403004C2403004C1D0300EC
:10D06000801D0300941D0300A81D0300BC1D0300C8
:10D07000D01D0300E81E0300741E03006C1F030094
:10D08000D83E0020AD3E0020AC3E0020401F0300F3
:10D090004C1E0300C81E0300EC1D0300201E0300ED
:10D0A000141F0300A41E030008B502F02FFC00B9F2
:10D0B00008BDBDE80840FBF749BB00BF70B55F4E37
:10D0C00033688CB06BB1044648F2FE000D46039005
:10D0D00019460822002305A8049304F07CF8012DCA
:10D0E00001D00CB070BD564BA4F119001D7007287B
:10D0F00000F29B80DFE800F02B5E869999999904F5
:10D10000504B51485149C01AC008000440F0030078
:10D11000FAF7C4FA31684FF47A7248F2FE0000233D
:10D120000831ADF82E2007900822012409A80893A1
:10D130008DF82C4004F04FF807AB1A46306803A96D
:10D1400001F06AFB0028CCD0FBF700FBC9E73D4BA0
:10D150003D483F49C01AC008000440F00300FAF7F8
:10D160009DFA002403221223694601A88DF8054088
:10D170008DF80420029302F0C7FA002858D13168D4
:10D1800000230831082248F2FE0409A8CDE907432C
:10D1900004F021F8009B98680A224121083004F02D
:10D1A00025F83068009B07AA03A901F0FDF90028C3
:10D1B00097D0C9E7234B24482649C01AC008000469
:10D1C00040F00300FAF76AFA0024032212236946AA
:10D1D00001A88DF805408DF80420029302F094FA1E
:10D1E00048BB009B98680A224121083003F0FEFFEB
:10D1F0003068009B184A03A901F0D6F900283FF4D3
:10D2000070AFA1E70F4B10481449C01AC0080004C2
:10D2100040F00300FAF742FA3068114A03A901F01E
:10D220004FFA00283FF45DAF8EE700221A7058E7EE
:10D23000FBF78CFAA3E7FBF789FAD2E7DC3E002084
:10D24000D83E0020242403004C240300AC1C03001F
:10D25000381D0300081D03008C1C0300D41C0300B0
:10D260009C1C030010B5047A012C0ED0022C0BD1AB
:10D27000134B14481449C01AC008000440F00300BE
:10D28000FAF70CFA114B1C7010BD0D4B0D4C1049E8
:10D29000E41AE408240444F003042046FAF7FEF9F3
:10D2A0000C4B186802F036FF08B1FBF74FFA204626
:10D2B0000949FAF7F3F9054B01221A7010BD00BFB6
:10D2C000242403004C24030044200300AD3E00202E
:10D2D00060200300D03E00208020030070B55A4A31
:10D2E00084B01021C020FBF779FA08B1FBF72EFAC1
:10D2F0000023012455484FF0A041032203E00642D9
:10D3000018BF41F825200133202B04FA03F603F55A
:10D31000E075F4D14FF0A0434C4AC3F80825002231
:10D32000C3F80C25FBF70AFD08B1FBF70FFA484AD2
:10D3300048480121FBF738FD08B1FBF707FA4FF425
:10D3400080410020FAF74AF908B1FBF7FFF9FAF734
:10D35000CBF840F2333204213F48FBF785F908B19E
:10D36000FBF7F4F9FBF7DCF908B1FBF7EFF93B4801
:10D3700002F092FA08B1FBF7E9F9002240F2666187
:10D380003748FBF71FFD08B1FBF7E0F9354C0822E1
:10D390000021204603F02AFF3349344B2160344AF0
:10D3A00063602046012102F033FF08B1FBF7CEF99C
:10D3B0002F4D6946286802F0D5FE0023694628688B
:10D3C0008DF8053002F0E4FE08B1FBF7BFF92949FA
:10D3D000286802F0F5FE08B1FBF7B8F9254A264B9C
:10D3E000029202A8039302F071FC08B1FBF7AEF9B8
:10D3F000224801F0E3FA08B1FBF7A8F9204B214CD1
:10D400002149E41AE408240444F003042046FAF70E
:10D4100045F9286802F07EFE08B1FBF797F920462F
:10D420001A49FAF73BF91A4B01221A70FBF768FA0E
:10D43000FAF702FD0028F9D1FFF75CFC0028F5D0CF
:10D44000FBF784F9F2E700BF5C3100200000E30144
:10D45000A9D0020028200300901F0020981F03007D
:10D46000B03E0020A43E002065D2020001CE0200A2
:10D47000D03E00203458002005CE02008DCE0200A0
:10D48000242403004C2403002C20030080200300EC
:10D49000AD3E00202DE9F041D0F8E03003F00F035D
:10D4A00003EB430300F120059B00EA180344C0F896
:10D4B000E82000F11C0784B004461A8D596A3846EA
:10D4C00003F0BEFD002876D0DFF8F0800390002640
:10D4D000D8F800308DF80060694620469847D4F8A7
:10D4E000E8301868FCF7A6FBD4F8E030C4F8E86030
:10D4F0000133C4F8E030D4F8E420D4F8E0309A42A4
:10D5000059D0D4F8E03003F00F0303EB43039B0042
:10D51000EA182344C4F8E8201A8D596A384603F003
:10D520008FFD002847D00390D8F800308DF80060B8
:10D53000694620469847D4F8E8301868FCF77AFB2B
:10D54000D4F8E030C4F8E8600133C4F8E030D4F82F
:10D55000E420D4F8E0309A422DD0D4F8E03003F043
:10D560000F0303EB43039B001D442344C4F8E8501E
:10D5700038461A8D596A03F063FDE0B10390D8F87C
:10D5800000308DF80060694620469847D4F8E830AE
:10D590001868FCF74FFBD4F8E030C4F8E8600133BA
:10D5A000C4F8E030D4F8E420D4F8E0309A4202D055
:10D5B0002046FFF76FFF04B0BDE8F081E43E002095
:10D5C0002DE9F04F734E32688DB0C2B1724F0D46E7
:10D5D000FC8B41882B784FF0000C8C42CDF814C0A6
:10D5E00013D0022B02D0032B05D0D3B10024204648
:10D5F0000DB0BDE8F08F0023D3F8E830FFDE4AF22B
:10D60000802420460DB0BDE8F08FB7F81CE0B0F8DC
:10D6100000C0E645E5D1032BE8D8DFE803F04692E9
:10D62000C94D6B685A6895798DF8185055798DF801
:10D63000195012798DF81A20FF25FE228DF81B5003
:10D640008DF81C205A68D2788DF81D205A6892787F
:10D650008DF81E205B685B788DF81F300CBBF9835A
:10D660000388BB834FF6FF733B82082206A94B4811
:10D6700003F0B1FD08224A49474803F0ACFDC0223F
:10D680002146484803F0B2FDC7F8E04001220B9460
:10D69000C7F8E440336840488DF8202008A998472F
:10D6A000A5E703F001FD0424A1E703F0FDFC00243D
:10D6B00020460DB0BDE8F08FD7F8E8301868FCF7C9
:10D6C000B9FAD7F8E0300133C7F8E030D7F8E420F2
:10D6D000D7F8E03000249A42C7F8E84086D0D7F85F
:10D6E000E030314803F00F0303EB43039B00F918CC
:10D6F00020333B440A8DC7F8E830496A03F0A0FCA8
:10D7000000283FF473AF0B90336823488DF8204016
:10D7100008A99847D7F8E8301868FCF78BFAD7F8CB
:10D72000E030C7F8E8400133C7F8E030D7F8E4202C
:10D73000D7F8E0309A423FF459AF1748FFF7AAFEF6
:10D7400055E7002302218DF820100B9308A91248F9
:10D75000164D9047BE69EC2303FB06F307EB030865
:10D760001D444446206A08B1FCF764FA0C34A54213
:10D77000F8D14046EC22002103F038FDEC2306FBF3
:10D78000037700242046BE61FC83C7F8E8400DB053
:10D79000BDE8F08FE43E0020E83E0020F03E00208F
:10D7A000D43F0020083F0020043F0020A83F002075
:10D7B0006B681B689F889B899F420CA928BF1F46E6
:10D7C00007F1290341F8183D05A8FCF7EBF90446D9
:10D7D00000287FF40CAF6B68DDF814801B68D3F869
:10D7E00008A008909AF800305A09032A40F0D9801E
:10D7F0009AF90120002AC0F20081FF22CDE901221E
:10D800000AF10209C3F3C103022B00F06581032B67
:10D8100000F05E81012B00F0748199F80030C3F3B1
:10D82000830343F0600388F8003099F8001099F8FA
:10D8300001308A1003F00F0302F0300243EA811333
:10D840001343022209EB020188F8013008EB0200C1
:10D8500003F0C1FC09F104099AF800305A0707D413
:10D8600099F8003088F806309AF8003009F101097B
:10D8700013F0030316BFD54A99F80030D35C88F83B
:10D88000073008F1080B08F118034FF010024FF0B1
:10D890000001584608BF09F10109009303F0A6FCF6
:10D8A00000981022002103F0A1FC9AF8013013F037
:10D8B000400FC3F3011300F08F80002B00F03E8176
:10D8C000022B00F0A981032B4FF0080240F0608189
:10D8D000BF4908F1100003F07EFC08AA0199BD4879
:10D8E00001F03AFE0446002800F02E814AF240245E
:10D8F0009AF8013003F0080203F0030B5B0755D5DB
:10D90000002A00F0B480BBF1000F48D1FF23494644
:10D91000022288F8183008F1190003F05CFC09F1C4
:10D920000201042208F1240009F1060903F053FC66
:10D930009AF8003013F0040B69D12820A9EB0A02F1
:10D94000BA1A92B29742A8F8042028D34946404414
:10D9500003F041FCB8F8043098F806205B449BB211
:10D9600003F12807112A5BBABFB2A8F8043000F00F
:10D970004B81DDF81480002C00F0D9804AF240235E
:10D980009C420FD1019B8DF82A30029B0B940322FD
:10D99000CDF82480ADF828708DF82B307AE6DDF8CC
:10D9A00014800B244046FCF745F920E6002A7BD082
:10D9B000BBF1020F00F08481BBF1030F00F077810F
:10D9C000BBF1010F00F0638149460098102203F07B
:10D9D00002FC09F11009ABE7022B584600F0FE806B
:10D9E000032B00F0E880012B00F0D980494610227B
:10D9F00003F0F1FB09F110097AE79AF80220110906
:10DA000002F00F020AF1030901910292FAE699F875
:10DA100000B00BF0F803F02BC1D10BF0030211237F
:10DA2000022A88F8063009F1010100F0C281032AB8
:10DA300000F0A781012A08F128004FF0020200F04F
:10DA4000948103F0C8FB09F10301022208F12A00C6
:10DA500009F1050903F0BFFB1BF0040F00F07A8108
:10DA60000023A8F82E3030204FF0080B66E7BBF1FA
:10DA7000020F00F06081BBF1030F00F05581BBF194
:10DA8000010F8CD10822494608F12000914403F08F
:10DA9000A2FB08AA02994F4801F05EFD002800F0A1
:10DAA0001F814AF2402443E7BBF1020F009800F0C7
:10DAB000DB80BBF1030F00F0CC80BBF1010F00F065
:10DAC000BC804946102203F086FB09F110092FE7BC
:10DAD0006023C8F80030BFE699F80030C3F3830331
:10DAE00043F0600388F8003019F8012B931003F01D
:10DAF000300343EA8213002288F80130A8F802209C
:10DB0000AAE64946602388F8003011F8012B9310EB
:10DB100003F0300302F00F021343022288F80130B1
:10DB200008EB020009F1030903F055FB94E6AB682A
:10DB3000B3F5044F08BF4FF4044423E71946584691
:10DB4000102203F053FBD3E608994A785846043173
:10DB5000D20803F040FB08994B7813F0070C3FF410
:10DB6000C7AEDB0808EB03004FF47F4290F808E0F3
:10DB700042FA0CF20B442EEA020E1B7980F808E000
:10DB8000497808EBD10113400A7A13430B72AFE6D0
:10DB9000494608F11000914403F01DFB9DE6022266
:10DBA0000D4903F018FB0822494608F11000914482
:10DBB00003F011FB9CE60222074903F00CFB08224C
:10DBC000034908F1100003F006FB91E6A4200300CE
:10DBD000F03E0020E83E0020AC2003001A467D49BC
:10DBE000039303F0F8FA039B7B491A4608F11300EC
:10DBF00003F0F1FA039B49461A4608F1160009F1B1
:10DC0000020903F0E8FA73E6022208F1040108F1C0
:10DC10002C0003F0E0FAACE61A46494608F116007B
:10DC2000039303F0D8FA039B6B491A4608F11300DB
:10DC300009F1020903F0CFFA4FE60222654903F029
:10DC4000CAFA0822494608F12000914403F0C3FAB9
:10DC50006EE602225F4903F0BEFA08225F4908F12E
:10DC6000200003F0B8FA63E65A465A4903F0B3FAC3
:10DC70005A46594908F1230003F0ADFA49465A467D
:10DC800008F1260009F1020903F0A5FA50E6494619
:10DC9000FF2388F8183011F8013B88F81930052265
:10DCA00008F1230009F1060903F095FA40E640F275
:10DCB000FF23A8F8183019F8013B88F8273037E619
:10DCC0004946FF2388F8183011F8013B88F81930CD
:10DCD000032208F1250009F1040903F07CFA27E684
:10DCE000089900984A780431D20803F074FA089928
:10DCF0004B7813F0070C3FF41BAEDB0808EB030076
:10DD00004FF47F4290F818E042FA0CF20B442EEAEE
:10DD1000020E1B7980F818E0497808EBD101134016
:10DD20000A7E13430B7603E608222C4908F12000F3
:10DD300003F051FAADE65A46274908F1230003F0F3
:10DD40004AFA49465A4608F1260009F1020903F049
:10DD500042FA9EE60222494608F12E0091444FF015
:10DD6000080B03F038FA3020E8E503F034FA99F8AC
:10DD700003301B0243F0F003A8F82A3009F104092C
:10DD80006AE699F801301B091B0243F4304343F063
:10DD9000F003A8F8283099F801301B0203F47063EF
:10DDA00043F4304343F0F003A8F82A3009F10209A4
:10DDB00052E699F801301B0243F0F00309F1020129
:10DDC000A8F8283008F12A0009F1040903F003FA41
:10DDD00042E600BFAC200300A8200300E83E00207C
:10DDE00018B1016809B1436813B94AF20E207047AF
:10DDF00030B5082283B004460C480D4D03F0EBF912
:10DE00000C4B62681A600021EC22284603F0EEF900
:10DE100002A8094B40F8043D0023EB83C5F8E83025
:10DE2000AB6103F0D5F803B030BD00BFD43F002094
:10DE3000E83E0020E43E0020C1D50200D34B1B6821
:10DE4000002B00F07581002900F086812DE9F04F4C
:10DE5000064691B0002800F09381272A40F2DC802A
:10DE600090F81080019200256023B8F1FF0F0C4656
:10DE7000D0F818A090F8119003958DF812508DF8F5
:10DE8000103000F00F82B9F1FF0F00F0CA802F466A
:10DE900045EA08158022EDB28DF811204FF0000BF5
:10DEA00049EA05058DF812500DF1130522786178C5
:10DEB00060881201D2B242EA11124FEA920C4CEA87
:10DEC000821252B2D3B2002800F0388101F00F0064
:10DED00013F03F0F04F1020100F04181022268704B
:10DEE0002B70A81803F077F90435A279112A40F0B5
:10DEF00022819DF8102042F004028DF81020E27972
:10DF0000402A00F0BA81FF2A00F0B081012A00F017
:10DF1000A6812A700135A2682AB9E2681AB9226975
:10DF2000002A00F00582B8F1FF0F00F06E819DF825
:10DF3000112042F04002236931688B4200F08B804F
:10DF4000002F00F0A58042F030038DF81130227EC2
:10DF5000FF2A00F0B580B9F1FF0F00F0958143F082
:10DF60000403206AB268904200F0C580BBF1000F44
:10DF700000F0578143F003038DF811309DF8103005
:10DF800013F0040340F008819846282604A96D1A6E
:10DF9000AAB2B61A2644304603F01DF9EC237C4A97
:10DFA00003FB0AFA02EB0A00D0F8E430D0F8E010E4
:10DFB0005B1A0F2B00F23281D0F8E410D0F8E43075
:10DFC000D0F8E47001F00F0103F00F0301EB410CF6
:10DFD00007F00F0E03EB43010AEB8C0C019BD0F80A
:10DFE000E47094440EEB4E0E0AEB8101283B0AEBE1
:10DFF0008E0A1144A3EB08035244CCF82460D0F8F5
:10E00000E86014621D4401370D85C0F8E470002EED
:10E0100000F06082002001E04AF2072011B0BDE864
:10E02000F08F01F11809494603AA01F009FA002806
:10E0300000F089812F469DF81220802142EA0812C3
:10E040008DF812208DF811104FF0000B4FF0FF09E2
:10E050000DF113052AE7207D317981427FF470AFFD
:10E06000E07CFF287FF46CAFFE297FF469AF606924
:10E07000484900EA010C706801408C457FF460AFAC
:10E08000E07DF17988423FF45EAF002F7FF45BAF13
:10E09000B3F17F4F03D1A38AFE2B00F0EC8142F055
:10E0A000100304F11001082228468DF811301544A0
:10E0B00003F091F8227E9DF81130FF2A7FF44BAFD8
:10E0C00043F00801B9F1FF0F8DF8111000F0018144
:10E0D00043F00C03227604F11901022228468DF840
:10E0E000113003F078F8A81C042204F1240103F095
:10E0F00072F8063542E794F82410327B8A427FF4A6
:10E1000035AF94F82310FF297FF430AFFE2A7FF457
:10E110002DAF204A616AF76811403A4091427FF47E
:10E1200025AFF27B94F8271091427FF41FAF21E7CF
:10E130004AF2802070472A700135E0E611F00F00A6
:10E140007FF4C6AE9DF81020002B40F0E98042F02D
:10E1500018028DF81020C8E64AF20E2070479DF88C
:10E1600010C022F03F02024328464CF0080C8DF804
:10E1700010C000F8012B022203F02DF80335B4E69D
:10E180004AF20E2011B0BDE8F08F00BFE43E00203F
:10E19000E83E002000FFFF00A379112B40F0BC8077
:10E1A000238D180A40EA03239BB223F00F0292B298
:10E1B0004FF2B001F0268A422E7000F0FD8003F489
:10E1C0007F43B3F5704F00F05C81638D1B029BB2FF
:10E1D000B3F5704F05F1010004F1280100F08581CD
:10E1E000022202F0F8FFE81C022204F12A0102F0E8
:10E1F000F2FF05352846022204F12E0102F0EBFF62
:10E20000023530264FF00808C0E6218948F2FE02A8
:10E21000914240F055819DF811208CE64AF2412050
:10E22000FCE6B0F17F4F0ED1A28CFE2A0BD143F059
:10E230000203022204F1260128468DF8113015440C
:10E2400002F0C9FF9AE643F00103082204F120011D
:10E2500028468DF81130154402F0BDFF8EE69DF87A
:10E26000102042F001028DF8102054E69DF8102095
:10E2700042F003028DF810204DE69DF8102042F088
:10E2800002028DF8102046E6218B48F2FE029142F0
:10E290003FF467AE2846102204F1180102F09BFFFC
:10E2A00010356BE601F1080B594603AA01F0C8F8D6
:10E2B000002800F09480B9F1FF0F00F020812F4674
:10E2C000AB469DF8125080228DF811204FF0FF08C8
:10E2D000E6E5A26922F0FF02B2F5007F00F0B68009
:10E2E000628B002AD6D1E269002AD3D1226A002AA1
:10E2F00000F0198132F07F42CCD12846627E43F093
:10E3000009038DF8113004F1230100F8012B0522D7
:10E31000063502F060FF31E628264FF0000835E6AA
:10E3200042F010028DF81020013505F8013CDCE5C3
:10E330006269002A7FF4F7AD9DF8113043F0400385
:10E340008DF8113003E603994A78802A00F0A48002
:10E350000746402A40F2DE80D5080F2D02F0070B59
:10E360000BD07119681C01314844C5F10F0202F04D
:10E3700023FF0399002840F0CD80705D254400FA0A
:10E380000BF02A7E02FA0BF2A0EB020BBBFA8BFB1E
:10E390004FEA5B1BB8F1FF0F91F8009040F08180CD
:10E3A000B9F1FF0F8DD100224FF0FF088DF8112039
:10E3B000C1460DF1120579E5618D0E0A46EA01218B
:10E3C00021F00F0189B291427FF4F9AE06F00F06F9
:10E3D00046EA0313F3226B702A7002350AE7039AA8
:10E3E0005378802B00F0B380402B40F29680DD08FC
:10E3F0000F2D03F007080BD0E91F681CC5F10F02B1
:10E400003144584402F0D8FE039A002840F0B1800D
:10E410007319254413F8081C2B7A01FA08F503FA3E
:10E4200008F3EF1AB7FA87F77F09B9F1FF0F92F8EF
:10E43000008000F0A080B8F1FF0F9DF8125008BFD7
:10E440004FF0000B3FF43FAF6DB221E5E269002AC7
:10E450007FF420AF226A002A7BD1626A32F07F42C9
:10E460005DD143F00B0394F827208DF8113001356E
:10E4700005F8012C82E542F0200304F11601022286
:10E4800012E6F223022268702B70A81804F12A0108
:10E4900002F0A1FE0435ADE691F8009007464FF07A
:10E4A000010B9DF8125045EA0815EDB28022B9F132
:10E4B000FF0F8DF812508DF811203FF4F5ACEFE40A
:10E4C0002846102204F1080102F085FE10359DF85F
:10E4D00011303CE5D0F8E420D0F8E0309A423FF427
:10E4E00099ADFEF7D7FF304698E5F1232B70022255
:10E4F00002F071FE638D1B0AEB7004357AE604F1BD
:10E50000180903AA4946304600F09AFF30B32F4657
:10E51000AB4648E74FF0000B3CE7074685E7628BC8
:10E52000002A7FF4B7AE94F82420002A7FF4E5AEE9
:10E530002846627E43F00A038DF8113004F125016C
:10E5400000F8012B0322043502F045FE16E50127F1
:10E550006BE7618B00297FF49DAECBE603994A7887
:10E56000802A7FF4F5AE91F8009007464FF0010B3A
:10E5700016E7002759E704F1180903AA494630466F
:10E5800000F05EFF38B1B8F1FF0F08BF4FF0000B8D
:10E590003FF409AF4FE503994A78802A7FF4D9AE5A
:10E5A0004FF0010BF6E600BF2DE9F047424C24780E
:10E5B00082B084B150B149B142B13BB11C78032C57
:10E5C0000ED04CF2071002B0BDE8F0874CF20E10EE
:10E5D00002B0BDE8F0874CF2801002B0BDE8F087D1
:10E5E000D3F80880DFF8D4A01D464FF0000980233F
:10E5F000064608F8083CA8F1300008F8079C28F8FF
:10E60000069C17460C4601F029FF3A22402308F8E1
:10E610002A2C08F8293C94E80F00A8F1280C8CE873
:10E620000F0097E80F00A8F1180787E80F00EB68C4
:10E63000BAF8000028F8049C0833C3F3072102024B
:10E6400041EA032342EA102228F8022C28F82C3C45
:10E65000EB6802AC423324F8023D604622464B464A
:10E66000102101F0CDFE4B4622463846102101F024
:10E67000C7FED5E90201083122464B4689B2083867
:10E6800001F0BEFEBDF80630BAF80020DB435BBAED
:10E6900028F8063CD5E90213A1F1300403F130015A
:10E6A000C5E90241531C30462946AAF8003001F062
:10E6B000BDFC02B0BDE8F087E03F0020E23F002053
:10E6C0002DE9F047504B1B7884B04BB310B309B31E
:10E6D00002B3082317460D46002206464FF00309F1
:10E6E00001A90DEB03008DF809208DF80890039324
:10E6F00001F00AF80446C8B1444B45484549C01AE0
:10E70000C008000440F00100F8F7C8FF204604B03C
:10E71000BDE8F0874CF20E14204604B0BDE8F08747
:10E720004CF28014204604B0BDE8F087019BD3F87A
:10E730000880852308F8070C28F8060C08F8083C20
:10E74000A8F1300001F08AFE3A22FF2308F82A2CB3
:10E7500008F8293C95E80F00A8F1280A8AE80F007C
:10E7600097E80F00A8F1180787E80F00019BDB6806
:10E7700048F8044C0833C3F3072242EA032301227A
:10E7800028F82C3C88F8002088F8012031464A46B9
:10E7900008F1020002F01FFD4A46711D08F1050054
:10E7A00002F019FD019BDB6804AD423325F80E3DF4
:10E7B00050462A462346102101F022FE23462A46CF
:10E7C0003846102101F01CFE019BD3E902010831FB
:10E7D0002A46234689B2083801F012FEBDF80230FD
:10E7E000DB435BBA28F8063C0199D1E90223303AB1
:10E7F00030333046C1E9022301F018FC04462046BC
:10E8000004B0BDE8F08700BFE03F002024240300EF
:10E8100074240300382203002DE9F047634C247868
:10E8200084B0002C00F0AE80002800F0A580002904
:10E8300000F0A280002A00F09F80002B00F09C8056
:10E840001D461B7C002B91464FF0000314BF28226D
:10E850001822884607464FF0030A01A902A803922E
:10E860008DF809308DF808A000F04EFF064600280C
:10E8700040F08E80019B9C68872304F8070C24F8E5
:10E88000060C04F8083CA4F1300001F0E7FD3A2240
:10E89000FF2304F82A2C04F8293C98E80F00A4F17F
:10E8A000280888E80F0099E80F00A4F1180989E802
:10E8B0000F00019BDB6844F8046C0833C3F30722A4
:10E8C00042EA032324F82C3C95E80F004FF0010C9A
:10E8D00084E80F0084F810C084F811C0524639460D
:10E8E00004F1120002F077FC524604F11500791D84
:10E8F00002F071FC2B7C73B16A8AA683130243EA8F
:10E90000122340F22122A261E3830822394604F156
:10E91000200002F060FC019BDB6804AD423325F867
:10E920000E3D40462A460023102101F069FD48466D
:10E930002A460023102101F063FD019BD3E9020167
:10E9400008312A4689B20838002301F059FDBDF884
:10E950000230DB435BBA24F8063C0199D1E902237B
:10E96000303A30333846C1E9022301F05FFB0646F6
:10E97000304604B0BDE8F0874CF20E16304604B0C5
:10E98000BDE8F0874CF28016304604B0BDE8F08751
:10E99000074B08480849C01AC008000440F00100AD
:10E9A000F8F77CFE304604B0BDE8F087E03F002079
:10E9B000242403007424030038220300074B1A7830
:10E9C000034622B130B1064A0020136070474CF272
:10E9D000801070474CF20E10704700BFE03F0020DF
:10E9E000DC3F00200349044B0020012208601A701C
:10E9F000704700BFDC3F0020E03F0020A74B1B78A2
:10EA0000002B36D0002831D081B37AB32DE9F04FF6
:10EA10001446D268072A95B00E46054602D98B885F
:10EA2000072B29D89E4B9F489F49C01AC008000455
:10EA300040F00100F8F7E0FF4CF2421302939B4BC9
:10EA40001E68002E00F0E181A16831F8063C1A0230
:10EA500042EA132221F8062C029B0094A1F108023D
:10EA600028463039B04715B0BDE8F08F4CF20E1093
:10EA700070474CF28010704714AF3A3227F8322DAD
:10EA800001F108093A4648460023102106F1180B07
:10EA9000D4F8088001F0B4FC3A465846002310210F
:10EAA00001F0AEFC3A460023A189A06801F0A8FC61
:10EAB000D4E90271BDF81E30DB439BB207F1080AAE
:10EAC000A1F108020320ADF81E30C4E902A22070B3
:10EAD000002B40F0858198F80020812A0ED8802AEA
:10EAE00080F09981013A032A00F29181D8F804302C
:10EAF0001BBAC8F8043000230293A0E7853A032A22
:10EB000000F285810B1F391DC4E9021398F800201B
:10EB1000853A0846032A00F25C82DFE812F05101D0
:10EB2000A20096000600DDF80C800022029204305C
:10EB3000043BC4E9020398F80020802A7FF47FAFE9
:10EB400000210322E3688DF839100EA809A98DF879
:10EB500038200F9300F0D8FD0746002840F05D8173
:10EB6000099BD3F808A081230AF8070C2AF8060CA1
:10EB70000AF8083CAAF1300001F070FC3A22402368
:10EB80000AF82A2C0AF8293C99E80F00AAF118097A
:10EB900089E80F00099BDB680833C3F3072242EAC8
:10EBA00003232AF82C3C337EFF2B00F050819BE896
:10EBB0000F00AAF1280B8BE80F00B8F804302AF8F0
:10EBC000043CB8F806302AF8023C099BE2689868D1
:10EBD000A16802F000FB099BDB6814AE423326F803
:10EBE000303D584632460023102101F009FC4846CA
:10EBF00032460023102101F003FC099BD3E90201F6
:10EC00000831324689B20838002301F0F9FBBDF81B
:10EC10002030DB435BBA2AF8063C0999D1E902238C
:10EC2000303A3033C1E90223284601F0FFF90028C9
:10EC30003FF405AF1B481A4B1D49C01AC008000419
:10EC400040F00100F8F72AFDF9E60431284601F00A
:10EC500055F9002800F008810022D4E9020302924D
:10EC600065E7318948F2FE02914240F0EC800C2BBE
:10EC70007FF65BAF0B49DFF828C07A7CA1EB0C0173
:10EC8000C908090441F0010102911037002A00F07F
:10EC900099814FF00C0ACDF80C8040E0E03F002055
:10ECA0002424030074240300B0200300DC3F002070
:10ECB000F8210300222925D10DF13C081022002162
:10ECC000404602F093FA07F108030FCB88E80F00E3
:10ECD000BB788DF83930FB7803F00F01C3F30013D4
:10ECE0008DF838108DF84C30FB88002B40F099805F
:10ECF00008AA284600F030FC002800F04581D4E93D
:10ED000002037A780AEBC20A1FFA8AFA9A45BFF41C
:10ED10000AAF00EB0A077A78002A00F051813978AF
:10ED20000329C7D1BB78002B00F04181FB785A063C
:10ED300040F13D811B0600F13A813A8A48F2FE0318
:10ED40009A4273D04FF0000C082229460BA8CDE957
:10ED5000093C02F040FABA7807F11001D20809A87C
:10ED600002F039FABB7813F0070118D0DB0814AAB7
:10ED7000D0184FF47F4C10F82C2C4CFA01F13B4486
:10ED800022EA01021B7C00F82C2CBA7814A800EBB4
:10ED9000D2020B4012F82C1C0B4302F82C3C7B686F
:10EDA00009A9002B47D0022328468DF8343001F002
:10EDB0001BF80028A3D089490298F8F76FFC9EE75A
:10EDC000874B88488849C01AC008000440F00100F9
:10EDD000F8F764FC4CF240130293D4E90203A6E670
:10EDE00080487F4EB8F802100092801B0A02C008CB
:10EDF00042EA1122000440F0010092B27B49F8F788
:10EE0000FDFE4CF24113029319E630462BE64CF21C
:10EE10004013029313E602938FE67248704B7449D5
:10EE20000BE70EA9284600F07DF968E771490298C2
:10EE3000F8F734FC63E7284601F090F800283FF427
:10EE40005EAF6D49F3E74CF2431202926FE648F26F
:10EE5000FE034AE90A3708222946AAF1200002F0F7
:10EE6000BAF9AAF1280BA8E618238DF839004FF05B
:10EE7000030209A90EA88DF838200F9300F044FC76
:10EE80000290002840F08880099B9A6888231746E2
:10EE900002F8070C22F8060C02F8083CA2F1300038
:10EEA00001F0DCFA3A22FF2307F82A2C07F8293C64
:10EEB0009AE80F000397283F87E80F0099E80F00B2
:10EEC0000497039FA7F1180C8CE80F00099B039986
:10EED000DB68029F01F8037C0833C3F3072242EA90
:10EEE0000323602221F82C3C01F8042C0F46CDF8B6
:10EEF00014C09AE80F004FF0020C87E80F000123BE
:10EF000087F810C07B7407F112000322294602F033
:10EF100062F9039F032207F11500691D02F05BF9F6
:10EF2000099B029FDB6804980DF1500A42332AF8CE
:10EF3000303D10213B46524601F062FA3B465246B4
:10EF40000598102101F05CFA099BD3E90201083110
:10EF50003B46524689B2083801F052FABDF82030DB
:10EF6000039FDB435BBA27F8063C0999D1E90223EA
:10EF7000303A3033C1E90223284601F057F80290B5
:10EF800018BBD4E90203D2E50899284600F020FA1C
:10EF90007A78D4E90203B5E61248114B1749C01A32
:10EFA000C008000440F00100F8F778FBE9E7DDE96C
:10EFB00002081349F8F772FB4CF243130293E0E79F
:10EFC000DDF80C8002980F49F4E70648044B0E491F
:10EFD000E5E74CF240120292A9E500BF8C21030044
:10EFE000242403007424030024210300E4200300EC
:10EFF0003822030070210300B8210300142203000B
:10F00000D021030054210300F82103002DE9F04131
:10F010000E4C4FF0FF0804F5C077A4F10C06002554
:10F0200004F8048C04F8035C2574204610220021A7
:10F03000183402F0DBF8BC4235713560F0D1044B76
:10F0400001221A700020BDE8F08100BFF03F0020CF
:10F050006C41002008B50E4B1B789BB1A8B10D4A3E
:10F06000136863B10C4B0D480D49C01AC008000469
:10F0700040F00100F8F712FB4BF2041008BD1060DD
:10F08000184608BD4BF2801008BD4BF20E1008BDAB
:10F090006C410020E43F0020242403006C24030082
:10F0A000642203001A4B1B78A3B170B32DE9F04121
:10F0B000184E3368834210D0174B18481849C01AAD
:10F0C000C008000440F00100F8F7E8FA4BF2051020
:10F0D000BDE8F0814BF28010704706F10C0406F594
:10F0E000C678FF27002504F8047C04F8035C257427
:10F0F000204610220021183402F078F8444535717A
:10F100003560F0D10020BDE8F0814BF20E10704761
:10F110006C410020E43F0020242403006C24030001
:10F1200064220300A44B1B7833B3002900F0FC8059
:10F130002DE9F04F91F800A0BAF10F0F87B016D863
:10F140004B78802B13D89D4F3B6898428B4616D046
:10F150009B4B9C489C49C01AC008000440F0010029
:10F16000F8F79CFA4BF2051007B0BDE8F08F4BF2B0
:10F17000071007B0BDE8F08F4BF2801070473B7A64
:10F180009A4500F0028197F82020924500F0FB801C
:10F1900097F838108A4500F0F48097F850008245BF
:10F1A00000F0ED8097F86840A24500F0E68097F8FF
:10F1B0008050AA4500F0DF8097F898600096B2452D
:10F1C00000F0D78097F8B090CA4500F0D08097F84B
:10F1D000C8C0E24500F0C98097F8E0E0F24500F0D1
:10F1E000C28097F8F880C24500F0BB8097F81061A4
:10F1F0000196B24500F0B38097F828610296B245B7
:10F2000000F0AB8097F840610396B24500F0A38010
:10F2100097F858610496B2454CD097F870610596FE
:10F22000B24508BF0F2446D0FF2B00F08C80FF2A88
:10F2300000F08B80FF2900F08A80FF2800F0898091
:10F24000FF2C00F0A480FF2D00F0A380009BFF2B7B
:10F2500000F0A180B9F1FF0F00F09F80BCF1FF0F1B
:10F2600000F09D80BEF1FF0F00F09B80B8F1FF0F12
:10F270005DD0019BFF2B00F09680029BFF2B00F0DE
:10F280009480039BFF2B00F09280049BFF2B00F0E7
:10F290009080FF2E08BF0F244AD0494B49484B4964
:10F2A000C01AC008000440F00100F8F7F7F94BF26B
:10F2B00004105EE70E2404EB440407EBC404083496
:10F2C00084F800A09BF8013063709BF8143023751C
:10F2D000251D10220021284601F088FF9BF80120FF
:10F2E0002846D2080BF1040101F075FF9BF80130AC
:10F2F00013F007003FF43DAFDB08E5184FF47F4201
:10F30000297942FA00F05B4421EA00021B792A7154
:10F310009BF8012004EBD204034022790020134320
:10F32000237107B0BDE8F08F4BF20E1070470A242E
:10F330003B7904EB4404013307EBC4043B7108340C
:10F340009BF800A0BCE70024F2E70124F0E70224C8
:10F35000EEE70324ECE70D24ADE70C24ABE70B2428
:10F36000A9E70A24A7E70924A5E70824A3E70724B7
:10F37000A1E706249FE705249DE704249BE70324D7
:10F3800099E7022497E7012495E7002493E70424F2
:10F39000CEE70524CCE70624CAE70724C8E70824FB
:10F3A000C6E70924C4E70B24C2E70C24C0E70D24F8
:10F3B000BEE70E24BCE700BF6C410020E43F002004
:10F3C000242403006C240300642203007C22030035
:10F3D000164B1B783BB390B189B110B5144B1A682A
:10F3E00082420FD0134B14481449C01AC0080004BD
:10F3F00040F00100F8F752F94BF2051010BD4BF246
:10F400000E1070470A78FF2A02D01A79013A1A7151
:10F410000024FF230B800C75081D1022214601F0EB
:10F42000E5FE204610BD4BF2801070476C41002075
:10F43000E43F0020242403006C2403006422030022
:10F440003F4B1B78002B78D0D8B1D1B1CAB12DE990
:10F45000F04FDFF800A183B00F460192DAF80020E8
:10F46000824211D03748384B3849C01AC0080004CE
:10F4700040F00100F8F712F94BF2051003B0BDE8B7
:10F48000F08F4BF20E1070479AF80480B8F1000F1D
:10F49000F2D04FF000094D460AF10C0414F8043C78
:10F4A000FF2B45D0237C002B42D014F8033C402B8B
:10F4B00038BF402313F0070218BF01224FEAD30BD5
:10F4C000ABEB02023946204603F0070601F074FE5A
:10F4D000D8B969004B190AEBC3035B4417F80B005A
:10F4E0001A7B4FF47F43334142401A420DD1B9F1A8
:10F4F000000F05D099F8012014F8033C9A4204D279
:10F50000134B01EB050903EBC9090135102D08F177
:10F51000FF3803D01834B8F1000FBFD1B9F1000F94
:10F52000AAD0019B0020C3F8009003B0BDE8F08F83
:10F530000135102DF2D01834B0E74BF2801070472F
:10F540006C4100206C240300242403006422030087
:10F55000EC3F0020E43F0020414B1B7883B160B1B9
:10F560005AB10F290FD810B43E4B1C6884420DD0FD
:10F570004BF205105DF8044B70474BF20E107047CC
:10F580004BF2801070474BF207107047187A884290
:10F5900047D093F8200088425FD093F83800884223
:10F5A00059D093F85000884253D093F868008842AD
:10F5B0004DD093F88000884247D093F89800884255
:10F5C00041D093F8B00088423BD093F8C8008842FD
:10F5D00035D093F8E00088422FD093F8F8008842A5
:10F5E00029D093F81001884223D093F8280188424B
:10F5F0001DD093F84001884217D093F858018842F3
:10F6000011D093F87001884208BF0F21B0D101EBEF
:10F61000410103EBC1030833002013605DF8044B84
:10F6200070470021F3E70E21F1E70D21EFE70C21F0
:10F63000EDE70B21EBE70A21E9E70921E7E70821DC
:10F64000E5E70721E3E70621E1E70521DFE70421FC
:10F65000DDE70321DBE70221D9E70121D7E700BF7E
:10F660006C410020E43F0020254A2649002310B4C5
:10F67000C2E90133D36013701361C2E90633136228
:10F6800013755362C2E90B33536382F828309363D6
:10F69000C2E91033936482F83C30D364C2E9153375
:10F6A000D36582F850301366C2E91A33136782F8C3
:10F6B00064305367C2E91F33C2E92433C2E92933F6
:10F6C000C2E92E330124C2F8843082F87830C2F8BF
:10F6D0008830C2F8983082F88C30C2F89C30C2F87A
:10F6E000AC3082F8A030C2F8B030C2F8C03082F836
:10F6F000B430C2F8C4300C7018465DF8044B704743
:10F70000704100206D410020474B1B78002B44D0F6
:10F7100000283FD000293DD003785A1E042A43D840
:10F720002DE9F0414678012E3AD8D0F804C0BCF15A
:10F73000000F3CD0023BDBB2032B9CBF3B4A52F88C
:10F7400023703B4B1A6994BFBC440027002A32D077
:10F750005A6A002A57D09A6B002A56D0DA6C002ACF
:10F7600055D01A6E002A54D05A6F002A53D0D3F8BD
:10F770008820002A51D0D3F89C20002A4FD0D3F8FB
:10F78000B020BAB1D3F8C420002A4AD04BF204000A
:10F79000BDE8F0814BF20E0070474BF280007047DD
:10F7A0004BF20700BDE8F0814BF2070070474BF2C7
:10F7B0000900EDE7082202EB8202920003EB020847
:10F7C0000D460446C8F810C08EB16368C8F80C3006
:10F7D000237888F800306378012B04D0D8F80430FF
:10F7E0001F44C8F80870C5F800800020D0E702F177
:10F7F0001001043219449818FAF7D4F90028E4D01B
:10F80000C8F81060C4E70122D5E70222D3E703223B
:10F81000D1E70422CFE70522CDE70622CBE7072276
:10F82000C9E70922C7E700BF6D410020A8220300F5
:10F8300070410020154B1B78BBB118B3144A821AD3
:10F84000C82A15D8134B10B5A3FB02431B0903EBC1
:10F850008303B2EB830F12D1044661B90020C4E9DF
:10F860000100E0602070206110BD4BF28000704705
:10F870004BF2100070474068FAF7DCF9EEE74BF204
:10F88000100010BD4BF20E00704700BF6D4100200C
:10F8900070410020CDCCCCCC70B370B4047804B3EC
:10F8A00043681A681AB35968632920D9154EA6FB14
:10F8B00001525209642505FB1212C2B9013CE4B29F
:10F8C00003EBC4040BE09A688AB1D968A6FB01C2B5
:10F8D0005209632905FB121209D908333AB9A34228
:10F8E000F1D1094A0023106070BC184670474BF2F2
:10F8F0000723184670BC7047034A0023106018465F
:10F90000704700BF1F85EB5138420020F8B5194FF2
:10F91000194E3B683268643313F1650F88BF642366
:10F920003B6022B392F800E0BEF1000F1FD0D2F886
:10F9300004C000240CE05CF835309847326801348C
:10F9400092F800E0E4B2A64511D9D2F804C03B68B1
:10F9500025B20CEBC50218465168B3FBF1F201FB6E
:10F960001233002BE7D00134E4B27445EFD300200A
:10F97000F8BD00BF3C420020384200202DE9F0478E
:10F980000B784769022B86B0044600F09080032B69
:10F9900044D0012B02D006B0BDE8F087BC4D2B68E7
:10F9A000002BF8D1BB4F636148F2FE0608222146C6
:10F9B0002C6003A80293019601F00DFC3B7C666964
:10F9C00002228DF81420002B40F0C58097F82430D7
:10F9D000002B40F0F48097F83830002B40F0FA808C
:10F9E0003B7C002B00F0458197F82430002B00F081
:10F9F000EE8097F83830002B00F0F4802046FFF7B7
:10FA000029FBA54AA54913680D680026013301A901
:10FA100020468DF804601360A847BCE70D464E6889
:10FA2000002F3ED1CB68052B3BD0D6F818E040F232
:10FA3000FF239E4500F0D980954A1379FF2B30D0E3
:10FA400002F1050A934F40F2FF2906F118080AE077
:10FA500001F0B2FB002800F0D8801AF8013BFF2B20
:10FA60001ED0D6F818E003EB83034FEA830CCE4593
:10FA70004FF01002414607EB0C00E9D1F369002B6F
:10FA8000E6D1336AB3F1807FE2D196F82430FF2BC0
:10FA9000DED10CF10D003844032206F12501D7E731
:10FAA0006E683046FAF7C6F806B0BDE8F087002F5A
:10FAB0007FF471AF06A9012301F8143D774B744D13
:10FAC0001B6898472046FFF7EDFA734A29791368B7
:10FAD0002F60013BFF2913601BD16B79FF2B27D1CE
:10FAE000AB79FF2B3FF457AF2B79FF22022BAA7182
:10FAF0003FF451AF6B79022B3FF44DAF654B0024BF
:10FB000003F128002146102283F8384001F06EFBF3
:10FB100041E76B79FF222A7153B1AB79002BDCD01E
:10FB20005C4B3946184610221F7401F05FFBD4E786
:10FB30002B79FF22012B6A71D2D0AB79012BD3D064
:10FB4000544B002403F114002146102283F8244072
:10FB500001F04CFBC4E7102201A9384601F02CFB50
:10FB600000287FF433AF8046F600AB191A79904530
:10FB700000F081805979884500F086809B7998450E
:10FB800000F08480FF2A00F08F80FF2900F0908031
:10FB9000FF2B7FF433AF42484FF0020909EB890392
:10FBA00007EB83079DF814303B74102201A92E4403
:10FBB00001F011FB06EB090383F804801EE7102215
:10FBC00001A9384801F0F8FA00287FF404AF4FF09B
:10FBD0000108C9E7102201A9314801F0EDFA002817
:10FBE0007FF4FEAE4FF00208BEE7F369002B7FF40E
:10FBF00023AF336A002B7FF41FAF736AB3F1B05F9A
:10FC000003D0B3F1807F7FF417AF01232A898DF8E9
:10FC10000530694601A88DF804300292FFF774FDA3
:10FC200000287FF43DAF009E6968F368716001F1C0
:10FC30002802283BC6E9022388884A888D79030276
:10FC400043EA10238B80130243EA1223112D4B80C9
:10FC500032D03A2D08D120463246FEF7CFFE4CF284
:10FC6000410398423FF497AE30460121FFF7E2FD91
:10FC700091E6984678E7002303EB830307EB8307BD
:10FC80009DF814303B74B9E60123F5E70223F3E74E
:10FC90008042002040420020884200207C42002018
:10FCA000684200205442002006484FF0000975E7E2
:10FCB00005484FF0010971E72046324600F0F8FB95
:10FCC000CDE700BF404200205442002018B1036835
:10FCD0000BB1436813B94CF20E00704770B53A4D42
:10FCE00082B00446F9F74EFFFFF7BEFC00F0BEFB02
:10FCF000FEF778FEFFF78AF910220021334801F061
:10FD000075FA334B2A79334960681860FF2A4FF03F
:10FD100000032B600B6024D12F4E6B79FF2B30D169
:10FD2000AB79FF2B35D10025294610222A4835749E
:10FD300001F05CFA29461022284886F8245001F088
:10FD400055FA29461022264886F8385001F04EFA16
:10FD50002268244B009268460193FEF741F802B0F6
:10FD600070BD6A79FF21297152B1AA791A4E002A11
:10FD7000D3D0194630461022337401F037FACCE75D
:10FD8000154E2B79FF22012B6A71C9D0AB79012B5B
:10FD900010D12B79FF22022BAA71C4D06B79022BD0
:10FDA000C1D00023194610220D4886F8383001F0E2
:10FDB0001DFAB8E7002319461022084886F82430B7
:10FDC00001F014FAACE700BF804200203C5800204C
:10FDD0007C42002088420020404200205442002003
:10FDE000684200207DF902002DE9F8433E4B1A6875
:10FDF000002A56D00D46C9B1C0B13C4C4769237C9E
:10FE0000002B46D194F82430A3B994F83830002B55
:10FE10004BD1267CB6B194F8243093B194F83830A5
:10FE2000002B49D04CF20400BDE8F8834CF20E00E0
:10FE3000BDE8F883102229462D4801F0BDF90028BD
:10FE4000E3D10126DFF8B080FF0008EB07031A7941
:10FE5000964233D059798E4239D09B799E4238D020
:10FE6000FF2A38D0FF293AD0FF2BDBD121484FF0B1
:10FE7000020909EB890304EB8304B8442B7C237447
:10FE8000C8442946102201F0A6F9002088F8046031
:10FE9000CAE71022204601F08FF90028B2D10646A9
:10FEA000D0E74CF28000BDE8F883102229461148C3
:10FEB00001F082F90028ACD10226C3E7002303EB4E
:10FEC000830304EB83042B7C23740020ACE7012321
:10FED000F5E70223F3E705484FF00009C9E70448B6
:10FEE0004FF00109C5E700BF7C42002040420020DE
:10FEF000544200206842002080420020144B1B68BE
:10FF000013B3F1B1E8B170B54369124CDB00E218EC
:10FF10001079FF2813D005330D460F4E1C4403E023
:10FF200014F8010BFF280AD000EB800006EB8000DC
:10FF30001022294601F040F90028F1D170BD0520BA
:10FF400070BD4CF20E0070474CF28000704700BF4D
:10FF50007C4200208042002040420020F8B5304B17
:10FF60001A68002A57D00E46002951D000284FD0D9
:10FF700044692C4DE4002B191879FF280AD12B195C
:10FF80005879FF282AD12B199879FF2833D14CF2C0
:10FF90000500F8BD244F00EB800007EB8000102225
:10FFA00001F00AF90028EAD12C440444FF2323710C
:10FFB0002B79984232D06B7998422FD0AB79984206
:10FFC0002CD000EB800007EB800700243846214648
:10FFD00010223C7401F00AF92046F8BD124F00EBE4
:10FFE000800007EB80001022314601F0E5F8002880
:10FFF000C9D10120D8E70C4F00EB8000314607EB58
:020000023000CC
:100000008000102201F0D8F80028C0D10220CBE7F0
:100010004CF20E00F8BD4CF28000F8BD0020F8BD97
:100020007C420020804200204042002038B50C4B2A
:100030001B688BB161B158B18A890C468968FDF79C
:10004000FDFE002105462046FFF7F4FB284638BD9B
:100050004CF20E05284638BD4CF28005284638BDC6
:100060007C4200206CDF70476DDF704772DF7047A5
:1000700073DF704778DF70477ADF70477CDF704747
:1000800069DF704730B589B0054610220021684607
:1000900001F0ACF8012404A810220021039500947B
:1000A0008DF8044001F0A2F82B880494112B8DF8F0
:1000B000144024D0262B0DD0102B28460ED0FF2321
:1000C0008DF8083000F076FD104B68461B689847A5
:1000D00009B030BD2B7A012B284605D102238DF8BB
:1000E000083000F067FDEFE713238DF81C3000F0B7
:1000F00061FD074B04A81B68984709B030BD28462E
:100100008DF8084000F056FDDEE700BF6C4300208C
:1001100068430020012801D00720704708B50D4A28
:100120000D4B52F8041B186800F03CFB70B90B4AE9
:1001300008490B48FFF79AFF08B1F8F707FB084B8F
:1001400023211878BDE80840FFF792BFF8F7FEFAC0
:10015000EDE700BFB01F0020784300201C430020C3
:10016000C01F002010B5012882B003D0072420460C
:1001700002B010BD6846FFF777FF06220446084626
:100180000DF1010101F027F8204602B010BD00BFBB
:10019000012811D14B797BB910B5084C2278204643
:1001A00063F3470200F8012B062201F014F8204601
:1001B000BDE81040FFF756BF07207047704300208E
:1001C000012801D00720704730B583B068460C463F
:1001D000FFF74AFFC0B99DF805009DF804309DF86F
:1001E00006509DF803109DF802206070A370FE2059
:1001F0009DF8013025702071FF250020E5706171A8
:10020000A271E37103B030BDF8F7A0FAE3E700BFD5
:100210002DE9F041036884B0002B00F0CC80012967
:1002200004D00724204604B0BDE8F0810D46694C97
:100230006949406815711560002220600B600092CA
:10024000FCF78AFB04460028ECD16846FCF7D2FC98
:1002500004460028E6D121460C2201A800F0C6FF82
:1002600001A9009A8DF8064040208DF807408DF8CE
:100270000550FFF705FF04460028D3D101460C22A4
:1002800001A800F0B3FF23260323009A8DF806503F
:1002900001A920208DF80460ADF80830FFF7F0FECA
:1002A00004460028BED101460C2201A800F09EFFA2
:1002B000009A8DF8044001A92846FFF7E1FE0446A4
:1002C0000028AFD1014604240C2201A800F08EFFC3
:1002D000424B009A8DF80A400DEB040124208DF862
:1002E00004608DF80B508DF80C50CDF80630FFF7F8
:1002F000C7FE0446002895D101460C2201A800F053
:1003000075FF4FF4807301A9009A0193A120FFF7B4
:10031000B7FE0446002885D16846FCF775FC044604
:1003200000287FF47FAF2E4D2E4EDFF8D0801422B0
:100330000021284600F05AFF112300272A48AB72FB
:1003400068602F8000F05AFF284B294A2881EA6014
:1003500039462B61A822304600F048FF0220254B89
:10036000307004202449F0704FF405707161C6F8B4
:1003700098001E602A896968C6F89470012305F107
:100380000A0086F8A470A6F89C70338286F8903034
:10039000C8F80050FFF772FEB8B92888FFF76AFE68
:1003A00070B905F10C00FFF767FE00283FF43AAF83
:1003B000F8F7CCF936E70E24204604B0BDE8F0810A
:1003C000F8F7C4F9D8F80050EBE7F8F7BFF9D8F818
:1003D0000050E2E7684300206C4300203200D40064
:1003E000544300208C420020B822030006002B005A
:1003F0000600180078430020C41F00207C43002022
:1004000070B41488250AE4B2C9B1067801293544CC
:10041000ADB2A1F102011ED04678344489B2A4B233
:10042000023014F47F4F02D00135E4B2ADB215F4BE
:100430007F4FE9D00134EDB2A4B20029E5D104EB3D
:100440000524A4B223B14FF6FF739C4208BF0024D9
:10045000148070BC70470021E3E700BF024B6022AC
:10046000C0E90023704700BF0000FF4070B50E4C8C
:10047000002504F1840610220021204624F8045CA3
:1004800024F8025CC4E9085500F0B0FE1022A01860
:1004900000212C3400F0AAFEB442ECD1034B01221F
:1004A0001A70002070BD00BF8843002080430020E8
:1004B00008B301B3FAB1D368082B19D98B88082B7C
:1004C00016D92DE9F0417F4F9668144673883A8813
:1004D000934286B00D4611D0BA8D9A421FD0B7F81C
:1004E00058209A422CD04CF2052006B0BDE8F0818D
:1004F0004CF2092070474CF20E20704710227249CE
:10050000381D00F059FE002875D17B88002B00F0C3
:10051000918032889A4200F08D807388DCE7102247
:1005200069496A4800F048FE00286DD1FB8D002B18
:1005300000F0918032889A4200F08D807388CEE777
:1005400010226149624800F037FE002865D1B7F8F3
:100550005A3013B132889A42C5D110225A495D48A7
:1005600000F02AFE38B1102205F10801594800F0C8
:1005700023FE0028B7D14FF00208B188E2680B02D1
:1005800043EA11239BB202F111019A42ADF80E1019
:100590004CD24CF24223A168CDF81080083AE260B8
:1005A00008312C2202FB0877A160D7E909020592E5
:1005B00000289AD070883188B288B6F806E04FEAF1
:1005C000002C4CEA102C080240EA1120110241EAEA
:1005D00012214FEA0E2242EA1E223080B180F280C0
:1005E000A6F802C0294632467D6A009404A8A847AE
:1005F00006B0BDE8F081102205F11801381D00F0A9
:10060000DBFD002881D088E7102205F118012F4872
:1006100000F0D2FD002889D090E7102205F11801E2
:100620002B4800F0C9FD002891D05CE725D94CF299
:100630004323B0E710222449274800F0BDFD40B114
:10064000102205F10801244800F0B6FD00287FF4CF
:1006500064AF804691E710221B49204800F0ACFDB2
:1006600040B1102205F108011C4800F0A5FD00284A
:100670007FF464AF4FF001087FE70DF10E02002315
:10068000102105F10800FFF7BBFE0DF10E0200235B
:10069000102105F11800FFF7B3FE0DF10E02002343
:1006A000A189A068FFF7ACFEBDF80E30013B9BB2FC
:1006B0004FF6FD72934288BF0023E26898BF4CF268
:1006C000412368E7844300203C580020B4430020C5
:1006D000E0430020F043002098430020C443002062
:1006E0006DDF704779DF70477DDF704764DF7047EB
:1006F0002DE9F04F83B004880C9EBDF83490B6F815
:1007000000A0002C39D09846002317468B4605469A
:100710001C4603E02A880134A24224DD6A6852F8AC
:100720002400019000220DF1030101A8FFF7DEFF74
:1007300020BB9DF80320BA42ECD13288B91803B32C
:1007400089452BDB42440DF1030101A80123FFF78A
:10075000CDFF98B931889DF803200A4432802A8859
:100760000134A242DADC43B13388013BA3EB0A0334
:100770009BB2FF2B12D808F80A30002003B0BDE866
:10078000F08F02310132894592B207DB328008F8DE
:1007900002B03288013292B23280D3E70C2003B02B
:1007A000BDE8F08F2DE9F04700231788138090F8FB
:1007B0002D3086B0144605460E46002B40F0FB80D7
:1007C000AA78002A40F0FD80EA78A2B1D91CB9428B
:1007D00000F2F3800221F154238801339BB20121FE
:1007E0002380F15423880B449BB22380F254238846
:1007F0000B449BB223806A68AAB1D91CB94200F2AB
:10080000DC80022192F90020F154238801339BB24D
:100810000A212380F154238801339BB22380F254B0
:100820002388013323802B89002B40F01B812B8AE6
:10083000002B40F02F812B8B002B40F043812B6A43
:10084000002B44D02288911DB94200F2B68019884D
:10085000052940F203816FF4486801EB080080B27B
:100860004FF27D3C604540F2F9805888052840F2FF
:10087000F5806FF4486E86441FFA8EFEE64540F21E
:10088000ED804FF6FF7C614504D0604502D0814287
:1008900000F2E4800521B1542288013292B2122183
:1008A0002280B1542288013292B222801988B15438
:1008B0003244090A51702288023292B222805B8847
:1008C000B35432441B0A53702388023323806B6A6B
:1008D000002B2FD09988B4F800C0881C0CF10202BC
:1008E0000244BA4269D8FE2867D8033106F80C10D2
:1008F0002288013292B2FF212280B1542288013233
:1009000092B222801988B1543244090A5170208869
:10091000023080B220809A8862B1996803930029DE
:1009200000F09C80304400F056FC039B9A8823889A
:100930001344238095F82C30002B40F08A802878CF
:1009400000283BD02B88012B00F08880228802F100
:10095000020CBC4531D8012804D16B780233134412
:100960009F422AD3BB1E9B1A06A99BB221F8083DC1
:1009700006EB0C00FFF7B8FE00BB2978BDF810208D
:10098000022900F0048168789042C0F0FB80934215
:10099000C0F0F8800921FE2A0FD82388501CF0549B
:1009A000238801339BB22380F154238801331A44F6
:1009B0002280002002E0082F23D80C2006B0BDE8DA
:1009C000F0870433BB42F8D804A8FFF78BFE002859
:1009D000F4D12388BDF810200321F154238801337A
:1009E0009BB219212380F154238801339BB2F11863
:1009F0002380F254120A4A70238802339BB2238068
:100A0000E2E604A8FFF76CFE0028D7D1138808227D
:100A1000CA54238801339BB21B222380CA542088E6
:100A2000013080B22080062208440DF1110100F04F
:100A3000D2FB23889DF8102006339BB212F0FE02F1
:100A400018BF01222380F254238801339BB22380F4
:100A5000B6E6D5F82880B8F1000F4CD1072006B0D3
:100A6000BDE8F08705F108080222CDE900474046BD
:100A700011463346FFF73CFE00289FD1CDE90047E1
:100A80004046334610220621FFF732FE00283FF48D
:100A9000CEAE93E705F11008CDE900474046334656
:100AA00002220321FFF724FE002887D1CDE9004769
:100AB0004046334610220721FFF71AFE00283FF474
:100AC000BAAE7BE705F11808CDE90047404633464A
:100AD00002221421FFF70CFE00287FF46FAFCDE94E
:100AE00000474046334610221521FFF701FE00283B
:100AF0003FF4A5AE62E7B8F804200232FE2A3FF6C2
:100B00005CAF23884FF000094FF0160A0132F2540F
:100B1000238801339BB2238006F803A02388013386
:100B20009BB22380B8F80020F2543344120A5A7062
:100B3000238802339BB22380B8F80410F0180A46C9
:100B400061B1D8F808301946002B87D000F043FB7C
:100B5000B8F80420238813449BB2238009F10109CB
:100B600095F82C205FFA89F94A4509EB49087FF688
:100B7000E6AEAA6A02EB8808B8F804200232FE2A20
:100B8000C4D91AE7012906D01A46082103E793427F
:100B9000BFF400AFF8E78342F6D302460821FAE635
:100BA000B8DF7047B9DF7047BADF7047BBDF704707
:100BB000A8DF7047A64B1A68002A46D0F0B5038814
:100BC0008BB000264FF6FF71722B044605960291FA
:100BD00000F0A38013D9742B74D046D3762B00F089
:100BE000B980772B09D19B4983880D88C0889D42A5
:100BF00003D14988814200F084810BB0F0BD112BF4
:100C00007ED023D9702B00F02B81712BF5D1914D23
:100C100080882988E3888842EFD14FF6FE718B42A5
:100C200002D069889942E8D1AB79012BE5D1002146
:100C300048F203404FF6FF738DF80C10A980A9719C
:100C4000854905902B60A9602BE07047102BD4D10B
:100C5000824803898B42D0D1A388038104F1090122
:100C60000622023000F0B7FAC7E77A4D8388288859
:100C7000E188012698428DF80C60BED14FF6FE70D7
:100C8000814202D068888842B7D14FF6FF70ADF834
:100C90000A10286000217048ADF80830A980A971B9
:100CA000A8606E490889984204F1040400F0788134
:100CB0000AAB002143F8104D0791049303A902A841
:100CC00090479AE7634983880888E588984294D1D9
:100CD0004888A84291D1A06801F10806B04204D327
:100CE000896801F5A051884287D3032048F2024168
:100CF000ADF80830ADF80A508DF80C000591D0E73A
:100D0000564C25898D427FF478AF07223146601C0E
:100D100000F06CFA258126706FE74E4D8388288895
:100D2000E18898427FF469AF4FF6FE70814203D0AC
:100D3000688888427FF461AFA87901287FF45DAFAD
:100D40000020ADF80A100221ADF808308DF80C0033
:100D5000A97135E03F4D83882988C08802269942D1
:100D60008DF80C607FF449AF4FF6FE71884203D0D6
:100D7000698881427FF441AFE668A968ADF80A004E
:100D8000A888ADF808308E4208BF20F0010001F5B8
:100D9000A06706BF80B24FF0010C4FF0000CBE42BE
:100DA00000F0CB8001F52067BE4200F0BA8001F56B
:100DB00070618E4200F0BC80BCF1000F40F0BB803F
:100DC00026490889984204F1040440F0DF800AAF04
:100DD000013147F8104D0791049703A902A89047E5
:100DE000AB88AA680692D8074FF4A062ADF81C2021
:100DF0007AD5AB68AA884FF4A06103F5A063ADF87B
:100E00001C109107069363D5AB68AA8803F520638D
:100E10004FF4A06152070693ADF81C104CD5AB6897
:100E2000AA8803F570634FF4A06106931307ADF829
:100E30001C103FF5E2AE3A4669882888FFF7B4FEF9
:100E400000287FF4DAAEAB8843F00803AB80D4E629
:100E500020440020084400202444002014440020A2
:100E600006AF574D31461022384600F0BFF92A88A8
:100E7000A088238A5349ADF824309042069117D0B8
:100E80005149B4F806C00E89ADF806C086420AD0B2
:100E9000232B3ED00223ADF826303A460DF1060151
:100EA000FFF77EFEA9E6232BF4D10B78012B30D17E
:100EB0000423ADF82630F0E73A4669882888FFF722
:100EC00073FE0028ABD1AB8843F00403AB80A6E7E8
:100ED0003A4669882888FFF767FE002894D1AB88D6
:100EE00043F00203AB808FE73A4669882888FFF712
:100EF0005BFE00287FF47DAFAB8843F00103AB803D
:100F000077E70320ADF80830ADF80A108DF80C0033
:100F1000C7E62389B3F5A06F15D20B23ADF82630B1
:100F2000BBE701F5706120F004008E4280B202D16F
:100F300020F0080080B2A88042E720F0020080B2D2
:100F40004FF0010C2EE74FF6FF739A4201D16B88E8
:100F500043B104233A460DF10601ADF82630FFF700
:100F60001FFE4AE63A460DF106010793ADF8203020
:100F7000ADF82630FFF714FEA8B100234FF6FF713D
:100F8000124A2960AB80AB71AA6036E60AAF002333
:100F900047F8104D0793049703A902A890471FE74D
:100FA0000AAB013186E6BDF82630002BE5D10123DE
:100FB000AB71A288BDF806302A806B801DE600BFA9
:100FC000084400200005320014440020244400207E
:100FD000F0B583B038B303682BB3012403464FF454
:100FE000C15520460DF1020201A98DF80640ADF869
:100FF0000450FFF7DDFD044690B90D4D0D4E0E4A2D
:1010000019680E4B11604FF6FF77701C0722AC80F9
:10101000AC71AB6021462F6000F0E8F83781347086
:10102000204603B0F0BD48F20E44204603B0F0BDA8
:1010300008440020144400202044002024440020C0
:10104000174B1B6823B100B129B948F20E40704715
:1010500048F28040704730B505884FF6FF739D42D7
:1010600083B01AD00F4B40881C88AC4206D14FF693
:10107000FE74A04206D05B88834203D048F205404C
:1010800003B030BD14460B466A460146284600931D
:10109000ADF80440FFF78AFDF2E748F20740EFE7BA
:1010A0002044002008440020154B1B681BB128B9C0
:1010B00048F20E40704748F28040704703884FF670
:1010C000FF72934219D010B40E4A418814889C4292
:1010D00006D14FF6FE73994207D053888B4204D055
:1010E00048F205405DF8044B704703239371418833
:1010F0005DF8044B0088FFF755BD48F20740704784
:10110000204400200844002008B5074B044613B1D2
:101110000021AFF30080054B1868836A03B198473C
:10112000204600F081F800BF00000000C422030048
:1011300070B50D4E0D4CA41BA4100025A54209D17D
:101140000B4E0C4C00F072F8A41BA4100025A54215
:1011500005D170BD56F8253098470135EEE756F8B1
:10116000253098470135F2E798210020982100208A
:10117000982100209C210020044B054A1B681B6A13
:10118000002B08BF1346D3F8EC007047C81F00209F
:101190002C20002082B001B901A942B14BB11378D3
:1011A0000B601278101C18BF012002B07047104667
:1011B000FBE76FF00100F8E730B50024A24201D14F
:1011C000002007E0035D01340D1915F8015CAB4206
:1011D000F4D0581B30BD10B5431E0A44914200D1D3
:1011E00010BD11F8014B03F8014FF7E70244034625
:1011F000934200D1704703F8011BF9E7034613F847
:10120000012B002AFBD1181A0138704749B1FF2A77
:1012100085BF8A2303600A704FF0FF3098BF01201A
:101220007047084670470000FEE700BFF8B500BFF2
:10123000F8BC08BC9E467047F8B500BFF8BC08BCB7
:101240009E467047FFFFFFFFFFFFFFFFFFFFFFFF0F
:10125000FFFFFFFF00000000000000000000D601BB
:1012600006010000D573020041740200D173020030
:10127000756172745F6C6F675F6261636B656E64EA
:1012800000000000102700207F00000090270020B1
:101290004261636B656E647320666C757368656428
:1012A00000000000617070000013030030130300A1
:1012B000E012030038130300401303004813030037
:1012C000501303005813030060130300202530322D
:1012D00078000000202020007C0000002563000032
:1012E0001B5B313B33316D0025734C6F677320649A
:1012F000726F70706564202825642925730D0A00BB
:101300001B5B306D00000000257300003C25733E20
:101310002025733A200000000D0A000000000000A4
:101320006813030070130300781303008013030095
:101330001B5B313B33306D001B5B313B33326D0047
:101340001B5B313B33336D001B5B313B33346D0032
:101350001B5B313B33356D001B5B313B33366D001E
:101360001B5B313B33376D006572726F720000009A
:101370007761726E696E6700696E666F00000000CB
:101380006465627567000000B02700206170705FBF
:10139000627574746F6E0000466174616C206572D2
:1013A000726F720053797374656D20726573657422
:1013B00000000000010006000000000010280020CE
:1013C0008D8902006170705F74696D657200000044
:1013D0000338FDD87047000052544320696E73747F
:1013E000616E636520616C726561647920696E6904
:1013F0007469616C697A65642E0000005254433A46
:1014000020696E697469616C697A65642E000000F8
:101410000000FFFFDEC0ADDEFE011EF1DEC0ADDE6E
:10142000FF011EF16D656D5F6D6E6772000000005B
:10143000303132333435363738394142434445460A
:101440006E72665F6673746F726167655F777269EB
:10145000746500006E72665F6673746F72616765B3
:101460005F65726173650000616464725F69735FD8
:10147000706167655F616C69676E656428705F663F
:10148000732C20706167655F6164647229000000DD
:10149000616464725F69735F77697468696E5F62C3
:1014A0006F756E647328705F66732C20706167655A
:1014B0005F616464722C20286C656E202A20705F46
:1014C00066732D3E705F666C6173685F696E666FF0
:1014D0002D3E65726173655F756E69742929000020
:1014E000705F667300000000257320636865636B9E
:1014F000206661696C656420696E20257328292047
:10150000776974682076616C756520307825782E4F
:1015100000000000705F617069000000705F64652A
:10152000737400006C656E00616464725F69735F60
:10153000616C69676E6564333228737263290000D9
:10154000616464725F69735F77697468696E5F6212
:101550006F756E647328705F66732C207372632CD2
:10156000206C656E29000000705F66732D3E705F11
:1015700061706900705F73726300000021286C6500
:101580006E202520705F66732D3E705F666C617300
:10159000685F696E666F2D3E70726F6772616D5F16
:1015A000756E697429000000616464725F69735F1D
:1015B000616C69676E6564333228646573742900F1
:1015C000616464725F69735F616C69676E656433DF
:1015D00032282875696E7433325F7429705F7372B4
:1015E00063290000616464725F69735F776974687E
:1015F000696E5F626F756E647328705F66732C200E
:10160000646573742C206C656E2900006E72665FD1
:101610006673746F7261676500000000736F7274A7
:101620006C69737400000000556E6B6E6F776E20EE
:101630006572726F7220636F6465000000000000C5
:10164000641703000100000070170300020000008F
:101650009017030003000000B4170300040000000B
:10166000C817030005000000DC1703000600000097
:10167000F01703000700000008180300080000002E
:101680002018030009000000381803000A000000B9
:10169000541803000B0000006C1803000C0000003D
:1016A000841803000D000000981803000E000000CD
:1016B000AC1803000F000000BC180300100000006D
:1016C000D018030011000000E81803001200000009
:1016D000F818030013000000101903008000000038
:1016E0002419030081000000481903008200000053
:1016F00064190300830000008019030084000000C7
:10170000A019030085000000C41903008600000032
:10171000EC19030090000000041A0300910000007F
:10172000241A030092000000441A03000082000003
:101730005C1A0300018200007C1A03000282000090
:10174000981A030000840000B41A0300018400000A
:10175000D81A030002840000041B03000384000065
:101760002C1B03004E52465F5355434345535300D1
:101770004E52465F4552524F525F5356435F484167
:101780004E444C45525F4D495353494E470000006B
:101790004E52465F4552524F525F534F4654444556
:1017A000564943455F4E4F545F454E41424C454478
:1017B000000000004E52465F4552524F525F494E64
:1017C0005445524E414C00004E52465F4552524FD6
:1017D000525F4E4F5F4D454D000000004E52465F38
:1017E0004552524F525F4E4F545F464F554E440044
:1017F0004E52465F4552524F525F4E4F545F5355C3
:1018000050504F52544544004E52465F4552524F3D
:10181000525F494E56414C49445F504152414D0040
:101820004E52465F4552524F525F494E56414C49C7
:10183000445F5354415445004E52465F4552524F07
:10184000525F494E56414C49445F4C454E475448BF
:10185000000000004E52465F4552524F525F494EC3
:1018600056414C49445F464C414753004E52465FF7
:101870004552524F525F494E56414C49445F444194
:10188000544100004E52465F4552524F525F444110
:1018900054415F53495A45004E52465F4552524F9C
:1018A000525F54494D454F55540000004E52465F1B
:1018B0004552524F525F4E554C4C00004E52465FBF
:1018C0004552524F525F464F5242494444454E00A2
:1018D0004E52465F4552524F525F494E56414C4917
:1018E000445F4144445200004E52465F4552524FBD
:1018F000525F4255535900004E52465F4552524F77
:10190000525F434F4E4E5F434F554E540000000010
:101910004E52465F4552524F525F5245534F5552B9
:10192000434553004E52465F4552524F525F4D4F12
:1019300044554C455F4E4F545F494E495449414CC4
:10194000495A4544000000004E52465F4552524FEE
:10195000525F4D555445585F494E49545F46414981
:101960004C4544004E52465F4552524F525F4D55D2
:101970005445585F4C4F434B5F4641494C454400EA
:101980004E52465F4552524F525F4D555445585F37
:10199000554E4C4F434B5F4641494C454400000077
:1019A0004E52465F4552524F525F4D555445585F17
:1019B000434F4E445F494E49545F4641494C45446C
:1019C000000000004E52465F4552524F525F4D4F4D
:1019D00044554C455F414C52454144595F494E493D
:1019E0005449414C495A4544000000004E52465F5C
:1019F0004552524F525F53544F524147455F4655EF
:101A00004C4C00004E52465F4552524F525F41507F
:101A1000495F4E4F545F494D504C454D454E5445DE
:101A2000440000004E52465F4552524F525F4645B9
:101A300041545552455F4E4F545F454E41424C45CF
:101A4000440000004E52465F4552524F525F494F8C
:101A50005F50454E44494E47000000004E52465FDD
:101A60004552524F525F4452565F5457495F455258
:101A7000525F4F56455252554E0000004E52465F3F
:101A80004552524F525F4452565F5457495F455238
:101A9000525F414E41434B004E52465F4552524FBA
:101AA000525F4452565F5457495F4552525F444E0D
:101AB00041434B004E52465F4552524F525F424C9B
:101AC000455F495053505F52585F504B545F5452DA
:101AD000554E4341544544004E52465F4552524F85
:101AE000525F424C455F495053505F4348414E4E10
:101AF000454C5F414C52454144595F455849535408
:101B0000530000004E52465F4552524F525F424CC6
:101B1000455F495053505F4C494E4B5F44495343D6
:101B20004F4E4E4543544544000000004E52465F20
:101B30004552524F525F424C455F495053505F509F
:101B40004545525F52454A45435445440000000014
:101B5000636C6F636B000000434C4F434B0000000D
:101B60004750494F5445000050525300554152547C
:101B700000000000554152544500000001000007DC
:101B8000082403001024030008000000F8230300C9
:101B90000824030008000000E8230300F8230300E2
:101BA000080000006E72665F73646800496E7375AA
:101BB0006666696369656E742052414D20616C6C84
:101BC0006F636174656420666F722074686520536A
:101BD0006F66744465766963652E00004368616EC4
:101BE0006765207468652052414D2073746172747A
:101BF000206C6F636174696F6E2066726F6D203048
:101C000078257820746F20307825782E0000000029
:101C10004D6178696D756D2052414D2073697A650B
:101C200020666F72206170706C69636174696F6E99
:101C300020697320307825782E00000073645F627D
:101C40006C655F656E61626C6528292072657475CC
:101C5000726E65642025732E00000000AC24030022
:101C6000B4240300080000006E72665F7364685F4E
:101C7000626C6500D8230300E8230300080000001D
:101C80006E72665F7364685F736F6300FF020000CB
:101C9000000000000000000000000001FF02000042
:101CA00000000000000000000000000253656E64A8
:101CB000696E67204E65696768626F757220536F41
:101CC0006C696369746174696F6E20746F207065EC
:101CD0006572210053656E64696E6720526F75747A
:101CE000657220536F6C696369746174696F6E20EB
:101CF000746F20616C6C20726F757465727320460E
:101D00004630323A3A32210050696E6720616C6C7D
:101D10002072656D6F7465206E6F646573207573D6
:101D2000696E6720464630323A3A31206164647207
:101D3000657373210000000050696E67207065654F
:101D4000722064657669636521000000476F742026
:101D500049434D5036204170706C69636174696FFE
:101D60006E2048616E646C6572204576656E7420E5
:101D70006F6E20696E746572666163652025700000
:101D8000095372632049507636204164647265734A
:101D9000733A200025303278253032783A253032B7
:101DA00078253032783A0000253032782530327884
:101DB0003A25303278253032780D0A0009447374A0
:101DC000204950763620416464726573733A20006E
:101DD0000950726F6365737320726573756C74203C
:101DE0003D2030782530386C580D0A0049434D505D
:101DF00036204D6573736167652054797065203DA9
:101E00002044657374696E6174696F6E20556E72DB
:101E10006561636861626C65204572726F72000073
:101E200049434D5036204D65737361676520547981
:101E30007065203D205061636B657420546F6F2086
:101E40004C6F6E67204572726F72000049434D50AF
:101E500036204D6573736167652054797065203D48
:101E60002054696D6520457863656564204572720C
:101E70006F72000049434D5036204D6573736167A2
:101E8000652054797065203D20506172616D6574E4
:101E900065722050726F626C656D204572726F7250
:101EA0000000000049434D5036204D657373616753
:101EB000652054797065203D204563686F20526528
:101EC000717565737400000049434D5036204D65AF
:101ED00073736167652054797065203D20456368A0
:101EE0006F205265706C790049434D5036204D6526
:101EF00073736167652054797065203D20526F755A
:101F000074657220536F6C696369746174696F6E74
:101F10000000000049434D5036204D6573736167E2
:101F2000652054797065203D20526F75746572206C
:101F30004164766572746973656D656E7400000046
:101F400049434D5036204D65737361676520547960
:101F50007065203D204E65696768626F7220536F1F
:101F60006C696369746174696F6E000049434D5018
:101F700036204D6573736167652054797065203D27
:101F8000204E65696768626F72204164766572747D
:101F90006973656D656E7400010000002020030008
:101FA000476F74204950204170706C696361746997
:101FB0006F6E2048616E646C6572204576656E7444
:101FC000206F6E20696E746572666163652025708E
:101FD000000000004E657720696E7465726661636B
:101FE000652061646465642100000000496E7465C9
:101FF00072666163652072656D6F766564210000AD
:10200000476F7420756E737570706F72746564209D
:1020100070726F746F636F6C206461746121000073
:10202000F9CC020090010000B03E00204170706CBD
:1020300069636174696F6E20737461727465642E74
:1020400000000000506879736963616C206C6179ED
:10205000657220636F6E6E65637465642E000000A8
:10206000506879736963616C206C61796572206472
:102070006973636F6E6E65637465642E00000000A3
:10208000506879736963616C206C6179657220694D
:102090006E20636F6E6E65637461626C65206D6F38
:1020A00064652E00000140FFFFFE0000FE8000007E
:1020B0005265636569766564206D616C666F726DEB
:1020C0006564207061636B65742C20776869636850
:1020D000206861732030782530386C58206279741C
:1020E00065732E0042616420636865636B73756D70
:1020F0002064657465637465642E20476F742030B6
:10210000782530387820627574206578706563743E
:102110006564203078253038782C203078253038A8
:102120006C580000476F7420756E737570706F7215
:1021300074656420526F7574657220536F6C6963A7
:1021400069746174696F6E206D6573736167652E64
:1021500000000000496E76616C6964207A65726FD8
:10216000206C656E677468206F7074696F6E2100F3
:1021700049676E6F7265204C696E6B2D4C6F6361A1
:102180006C207072656669782100000043616E6E94
:102190006F7420616464206E657720616464726589
:1021A0007373212041646472657373207461626C7F
:1021B000652066756C6C210043616E6E6F742072D1
:1021C000656D6F76652061646472657373210000CC
:1021D000507265666978206F7074696F6E206861EF
:1021E0007320696E636F72726563742070617261CF
:1021F0006D6574657273210043616E6E6F74207338
:10220000656E64207061636B6574206275666665D7
:10221000722100004661696C656420746F20616CF6
:102220006C6F63617465207061636B6574206275A7
:1022300066666572210D0A004661696C65642074EA
:102240006F20616C6C6F63617465207061636B6596
:1022500074206275666665722100000069636D70A6
:10226000360000004E6F20636F6E746578742074C2
:1022700061626C6520666F756E642E004E6F207013
:102280006C61636520696E20636F6E74657874207D
:102290007461626C652E0000636F6E746578745FA4
:1022A0006D616E61676572002800000030000000FB
:1022B00030000000340000004950763649434D504C
:1022C00000000000CC1F00204300504F534958002D
:1022D0002E00002020202020202020202828282810
:1022E00028202020202020202020202020202020E6
:1022F0002020208810101010101010101010101036
:102300001010100404040404040404040410101045
:1023100010101010414141414141010101010101F1
:10232000010101010101010101010101010110107F
:1023300010101010424242424242020202020202C5
:102340000202020202020202020202020202101051
:10235000101020000000000000000000000000003D
:10236000000000000000000000000000000000006D
:10237000000000000000000000000000000000005D
:10238000000000000000000000000000000000004D
:10239000000000000000000000000000000000003D
:1023A000000000000000000000000000000000002D
:1023B000000000000000000000000000000000001D
:1023C000000000000000000000000000000000000D
:0823D000000000000000000005
:1023D8002DAD02000000000081B2020000000000E4
:1023E8008DAB020000000000A9B20200000000004E
:1023F8009DCB020000000000A9CC020000000000F4
:08240800EDA902000000000034
:102410001C220020E4220020EC22002024220020A4
:0424200018000000A0
:10242400581B030000000000601B030000000000B4
:10243400681B0300000000006C1B03000000000088
:10244400741B030000000000A41203000000030337
:102454008C13030000000000C413030000000000FC
:10246400501B030000000000982203000000030337
:102474005C22030000000303241403000000000096
:102484000C16030000000303A41B03000000030355
:10249400681C030000000303801C03000000030306
:0824A4001C16030000000000FB
:0824AC008500030000000000A0
:1024B4006412030000000000701203007C1F00205F
:0824C4007C4DFF7F01000000C8
:1024CC000000000000200040000000000020004040
:1024DC000000000000000000FF0000000090D0038E
:1024EC00001001401100040020000300BDD00200C8
:1024FC001B000300BDD002001A000300BDD0020077
:10250C0019000300BDD00200344300201F0000005E
:10251C000000000000000000FF0000002018010077
:10252C00CC1F002000000000000000000000000094
:10253C00000000000000000000000000000000008F
:10254C00000000000000000000000000000000007F
:10255C00000000000000000000000000000000006F
:10256C00000000000000000000000000000000005F
:10257C00000000000000000000000000000000004F
:10258C0000000000430000000000000000000000FC
:10259C00000000000000000000000000000000002F
:1025AC0000000000430000000000000000000000DC
:1025BC00000000000000000000000000000000000F
:1025CC0000000000430000000000000000000000BC
:1025DC0000000000000000000000000000000000EF
:1025EC00000000004300000000000000000000009C
:1025FC0000000000000000000000000000000000CF
:10260C00000000004300000000000000000000007B
:10261C0000000000000000000000000000000000AE
:10262C00000000004300000000000000000000005B
:10263C00000000000000000000000000000000008E
:10264C00000000004300000000000000000000003B
:10265C00000000000000000000000000000000006E
:10266C00000000000D120300951103000000000093
:10267C00D2220300D0220300D1220300D122030076
:10268C00D1220300D1220300D1220300D122030066
:10269C00D1220300D1220300D1220300FFFFFFFF50
:1026AC00FFFFFFFFFFFFFFFFFFFF00000100415393
:1026BC004349490000000000000000000000000039
:1026CC00000000000000000000000000000041536A
:1026DC004349490000000000000000000000000019
:1026EC0000000000000000000000000000000000DE
:0826FC002572020001720200C8
:1027040000000000000000007D9B020000000000AB
:0427140000000000C1
:04000003200072B5B2
:00000001FF
